:020000041102E7
:1000000003B40148019001BD4539FF1F03B4014805
:10001000019001BDE927000003B40148019001BD32
:100020001D27FF1F03B40148019001BDADAE0000C4
:1000300003B40148019001BD456B010003B40148C0
:10004000019001BD0189000003B40148019001BD88
:10005000C53F000003B40148019001BDE94C010017
:1000600003B40148019001BDC95C010003B401481B
:10007000019001BDCD4C010003B40148019001BDC8
:10008000F54E010003B40148019001BD434D01004C
:1000900003B40148019001BDC51D000003B401482F
:1000A000019001BD154D010003B40148019001BD4F
:1000B0002526000003B40148019001BD8B520100C8
:1000C00003B40148019001BDB352010003B40148DB
:1000D000019001BD6189000003B40148019001BD98
:1000E000691F000003B40148019001BD5D170000C5
:1000F00003B40148019001BD3D4B010003B4014828
:10010000019001BD5952010003B40148019001BDA5
:100110005125000003B40148019001BD014C0100CC
:1001200003B40148019001BD594F010003B40148D7
:10013000019001BD1D4B010003B40148019001BDB8
:100140008D12000003B40148019001BD4D1F000055
:1001500003B40148019001BD5522000003B40148D9
:10016000019001BDDD52010003B40148019001BDC1
:100170001D4D010003B40148019001BD810E000036
:1001800003B40148019001BD017F000003B40148A0
:10019000019001BDE117000003B40148019001BDC9
:1001A0007918000003B40148019001BDD94901004C
:1001B00003B40148019001BDE928000003B40148DF
:1001C000019001BD5549010003B40148019001BDF2
:1001D0004551010003B40148019001BDC92600004A
:1001E00003B40148019001BDD536FF1F03B4014897
:1001F000019001BDE1AC000003B40148019001BDD4
:100200000124000003B40148019001BD1DBC0000A1
:1002100003B40148019001BD6DBC000003B4014866
:10022000019001BD0D52010003B40148019001BDD0
:100230003555000003B40148019001BD056A000076
:1002400003B40148019001BDED4A010003B4014827
:10025000019001BDA54F010003B40148019001BD0B
:100260008552010003B40148019001BD5D38FF1FB4
:1002700003B40148019001BDA930FF1F03B4014838
:10028000019001BDF94C010003B40148019001BD8A
:10029000C521000003B40148019001BD291C0000E4
:1002A00003B40148019001BDC94A010003B40148EB
:1002B000019001BD851F000003B40148019001BDFC
:1002C000090E000003B40148019001BD114701006F
:1002D00003B40148019001BD1131FF1F03B401486F
:1002E000019001BD350E000003B40148019001BD2D
:1002F000B538FF1F03B40148019001BDB30E0000E3
:1003000003B40148019001BD810E000003B401480F
:10031000019001BDD137FF1F03B40148019001BD19
:100320000938FF1F03B40148019001BDA537FF1F25
:1003300003B40148019001BD293AFF1F03B40148ED
:10034000019001BD4D3AFF1F03B40148019001BD6A
:10035000B54C010003B40148019001BD45500000B7
:1003600003B40148019001BDDD30FF1F03B4014813
:10037000019001BDD1A5000003B40148019001BD69
:10038000A946010003B40148019001BD594DFF1F6A
:1003900003B40148019001BDC9A9000003B401489C
:1003A000019001BD3141FF1F03B40148019001BD1F
:1003B000EDA5000003B40148019001BD553AFF1FAF
:1003C00003B40148019001BD2D38FF1F03B401485B
:1003D000019001BDC13AFF1F03B40148019001BD66
:1003E000F133FF1F03B40148019001BDB14E00007D
:1003F00003B40148019001BD3D18000003B4014859
:10040000019001BD2146010003B40148019001BDE6
:100410002124000003B40148019001BD75A900002A
:1004200003B40148019001BD9DA9000003B4014837
:10043000019001BD3543FF1F03B40148019001BD88
:10044000E134FF1F03B40148019001BD055E0000C7
:1004500003B40148019001BD8D35FF1F03B401486D
:10046000019001BDE548000003B40148019001BDC1
:100470002951010003B40148019001BDD91B0000BE
:1004800003B40148019001BD111FFF1F03B40148CF
:10049000019001BD391FFF1F03B40148019001BD48
:1004A0005147010070B5514A8AB0012800D1504A25
:1004B0004301504802AC1D18287E00280AD0842031
:1004C0008058C3B2002002E016782654401C98429F
:1004D000FADB04E0107D012310786A461072E869A7
:1004E000002807D06846017608A807940370E969D8
:1004F00006A888470AB070BDFEB5044642013D48D3
:100500003A4D1318805C191D00282AD0187E002847
:1005100027D0987E002824D00878022821D1888806
:100520004A888E68801A82B2102A01D9102201E00E
:10053000002A02D0012C17D01DE0012008700020F5
:1005400048808880D869002806D02B4A6D4607CAA3
:1005500007C5D96968468847002C03D01920FFF7E2
:100560004FFDFEBD0820FAE7214D04E04888431CFA
:100570004B80305C28701046521E92B20028F5D194
:10058000FEBD1B4880680007000F062812D006DC5D
:1005900002280AD004280DD10121012082E7072872
:1005A00005D00C2806D10221F7E70120A4E7104866
:1005B0004030C06B70470D4880680007000F062868
:1005C00012D006DC02280AD004280DD10121002017
:1005D00068E7072805D00C2806D10221F7E700209C
:1005E0008AE702484030C06B70470000004000407E
:1005F000009000401C52FF1F0C7A021110B5FFF74B
:1006000005FD022805D0072805D0122800D10220B8
:1006100010BD142010BD224904200A6B521C0A632D
:1006200010BDF8B500260C460D46074640341FE0C5
:10063000607CC1004A1953686A5C002801D001211E
:1006400000E000213846FFF7D9FF002802D0012141
:100650002176F8BD607CC00040194660607C401C7B
:100660006074207C401E20740D48016A491C0162A0
:10067000207C0028DCD166742676F8BD084A5C210F
:1006800041435C3A10B589185822525C012A05D1C1
:10069000FFF7C7FF0248816A491C816210BD000054
:1006A0006877FF1F10B504F019FE0621002005F041
:1006B00095FD0320FFF7B0FC032212020421402025
:1006C00005F0AAFD0120FFF7A7FC0223034AFE2143
:1006D000402005F045FC02F01FF910BDEC4EFF1F55
:1006E000F8B5D449D24A002004464A608300401C31
:1006F000D450FF28FADD4868CF4A014680318A602D
:100700006E22C262CD4A1278002A01D07F22C262D4
:100710000A220265CA4A13788363CA4BC3611578FB
:100720001023022D08D01578012D05D01578032D42
:1007300002D01578042D00D10362C34D45611925FF
:10074000AD0185613725CD6036272826C76308258A
:10075000466405644F6032270F603B27CF63412713
:10076000CF6439274031E0C132274F6002274F6103
:1007700042270831E0C11E274F60CE608D600526FC
:100780004E6142260E615A2660390E614D613C254C
:100790008D61AF25ED000560AC4D05631578022D28
:1007A00009D01578012D08D01578032D07D01578BC
:1007B000042D06D007E0152504E0436003E00E2574
:1007C00000E00C254560FF252D358560C560FF25BF
:1007D000F53505619E4D85647D25ED009D4ECD6707
:1007E000C66445629C4D85627325C56506254565D1
:1007F0008565C51D0826F93502272E6047664B27FB
:10080000FF0087660927C766944F07674667BE10D3
:100810008467C667924F8F4E3E601678022E09D0CD
:100820001678012E0AD01678032E0BD01278042ADF
:100830000CD00EE01A22CA61212205E01422CA61FE
:10084000182201E01322CB610A6202E00E220B6241
:10085000CA617F4A8A627D22D2008A6764224A6224
:100860000522CA6202220A63C8228C634A633821C5
:1008700069607C4929647C49A9614B21C900E9610F
:1008800074497B4A643929627D2109016962EC66F9
:100890001E212C67A9667149A965E9658910296639
:1008A000696469677149EA67A9677249FF308130F5
:1008B00006C00160FF21F531416081606F486E49DB
:1008C0005B4A81606E49803A11616C496D4A8031A2
:1008D0008A626D4ACA626D4A82616D4AC2626D4A1D
:1008E000026366486C4A403842636C4AC2636C4A91
:1008F000CA616C49816361496B48403188616C49C8
:100900006A4888605D486B4A803842606A4A426340
:100910006A4A0A626A49816058496A48C039C860AF
:10092000FFF780FB0120FFF783FBF8BDF3B5074617
:10093000654881B0C169654A1140FF310931C16123
:10094000002613E000252C461120FFF777FB5E48B8
:10095000406A8007800F610088402843641CE4B22D
:100960000546102CF0D301C7761CF6B202988642D9
:10097000E8D3FEBD10B52F4C607800280AD10421C1
:100980005348FFF7D3FF524804211030FFF7CEFF42
:100990000120607010BDF0B500248BB00D460646F6
:1009A000102902D901200BB0F0BDFFF7E3FF484941
:1009B00000200A5C401C1419C0B21028F9D3002C86
:1009C00003D0102D03D90B20EDE70E20EBE74148B3
:1009D0003F4C0023006802A91034E25CC75C7A40F7
:1009E000CA545B1CDBB2102BF7D306AA3848FFF7BA
:1009F0002BFB102D00D910252A4606A93046FFF7FB
:100A000029FBFFF72DFB216840182060FFF728FB2A
:100A1000616840186060FFF723FBA1684018A06080
:100A2000FFF71EFBE1684018E0600020BBE7000014
:100A30000004FF1F0851FF1FB07BFF1F744FFF1FF3
:100A40004A0AFF1F3A07000080C3C9019A0200004A
:100A500050C30000280A00006A180000204E000061
:100A6000F009FF1F0040001168100000DC050000C5
:100A700040420F0010270000953FFF1F0001FF1F9D
:100A8000F922FF1F7143FF1F5D46FF1F611FFF1FFC
:100A9000F520FF1F7D1FFF1F7D2CFF1FD52BFF1F84
:100AA000194CFF1F3D4AFF1F7D060211B526FF1F8F
:100AB0000002FF1F0D3CFF1FE93DFF1F2D3DFF1FE3
:100AC000C93BFF1FE526FF1F40F0004000FEFEFF70
:100AD0003476FF1F0052FF1F0A7802708A78427036
:100AE0004A88120A82700979C170042070470A7816
:100AF00002700988090A41700220704710B500226F
:100B00000EE093005B189C7804705C88521C240AE9
:100B100044701C7984709B88D2B21B0AC370001D7C
:100B20000B789342EDD81806800D10BDF8B50D4630
:100B300006464978012031700024761C16E0697859
:100B4000012917D01221614349198A7832704A88E5
:100B5000871C120A7270B61C10223046091DFFF75E
:100B600079FA1037B8B21036641CE4B22978A14281
:100B7000E5D8F8BDA10049198A7832704A88871CE7
:100B8000120A7270B61C02223046091DFFF762FA83
:100B9000BF1CB8B2B61CE7E710B50C460978017067
:100BA0002188090A41706288211D801CFFF752FAD2
:100BB0006088801C80B210BD10B50C4609780170A9
:100BC0002188090A4170A17881706188090AC17081
:100BD000A288A11D001DFFF73DFAA088001D80B26C
:100BE00010BD10B50C460A88891CFFF733FA20881F
:100BF00010BD10B50B788A7802705343DCB22246E0
:100C0000401C091DFFF726FA601C10BD10B50B78BB
:100C10008A7802705343DCB22246401C091DFFF75C
:100C200019FA601C10BD10B50C460A88891CFFF724
:100C300011FA208810BD10B50C460A88891CFFF7F0
:100C400009FA208810BD7FB515460446022901D057
:100C5000102903D1022B04D0102B02D0002004B0A5
:100C600070BD994202D10A46294607E0102969461B
:100C700007D000F00DF8102269462846FFF7F6F974
:100C8000EDE7104600F004F8102269462046F5E72B
:100C900070B50C4605000CD0002C0AD01022064975
:100CA0002046FFF7D7F92878207368786073012011
:100CB00070BD002070BD00009C7B021110B50B467A
:100CC0000122024901F01AFD10BD0000D90A0211EB
:100CD00070B5064608880C46172812D30B46032227
:100CE0000949304601F00AFD050008D1074920886E
:100CF0000988884200D20146304600F0B7F92846FC
:100D000070BD022070BD0000EF0A02113051FF1FBC
:100D100010B500231922194601F0F0FC10BD0000A7
:100D200010B50A78002A05D00B460722024901F0C7
:100D3000E5FC10BD022010BDFD0A021110B54A7875
:100D4000012A01D0022A08D10A78002A05D00B46D0
:100D50000522034901F0D2FC10BD022010BD0000A5
:100D60002D0B021101494000085A70472E51FF1FF8
:100D700010B50B461B22024901F0C0FC10BD00005B
:100D8000990B021101491720088070472E51FF1F4F
:100D90000098022B01D0042070471178527812027B
:100DA00089180180002070470098012B01D0042091
:100DB0007047117801700020704770B5049C1E4682
:100DC0001546062B1BD36978287809024018208025
:100DD000E978A87809024018608002222271291D52
:100DE000601DFFF737F9B61FB2B22281F02A06D88C
:100DF0002046A91D0A30FFF72DF9002070BD042000
:100E000070BD0098042B01D00420704753781178EE
:100E10001B02C91801809178D2781202891841808A
:100E200000207047F8B584890D460646002C26D070
:100E3000B2681778380620D50C2C20D90C3CA4B207
:100E40001019009001217088234601F0BFFA002894
:100E500011D0022028707806C00F6870B806800E86
:100E6000A870641E2004000CA88001D0B068401C4B
:100E7000A8600020F8BD0120ECE70020EAE701208F
:100E8000F8BD10B502981146042B14D34C780A789B
:100E9000240212190280CC788A7824021219428026
:100EA0001B1F9AB28280F22A05D8801D091DFFF708
:100EB000D1F8002010BD042010BD0098042B01D0F3
:100EC00004207047537811781B02C918018091786B
:100ED000D2781202891841800020704710B502981C
:100EE0001146062B03D0142B03D0042010BD022280
:100EF00000E0102202714B780A781B02D21802809F
:100F0000CB788A781B02D21842800279401D091DD5
:100F1000FFF7A0F8002010BD30B5039CD80718D10A
:100F2000D805010E022914D30B488088814210D8BD
:100F3000F6200155002008E0557813782D025B1942
:100F40004500401C6353C0B2921C8842F4D3002079
:100F500030BD042030BD00002851FF1F0098022B37
:100F600001D004207047117852781202891801804C
:100F70000020704770B5144602460498022B18D31F
:100F8000667825783602AD1905800546E0352A7663
:100F90006976002A0BD0E8219B1E9AB242808A42D1
:100FA00007D8A11C001DFFF755F8002070BDF421E3
:100FB000F2E7042070BD000010B50B46172202496D
:100FC00001F09CFB10BD0000B90B021110B50B46DF
:100FD0000D22024901F092FB10BD0000E30B02114B
:100FE00010B50A78002A05D00B461122024901F0FB
:100FF00085FB10BD022010BDF30B021110B50A785D
:10100000002A05D00B460922024901F077FB10BDEA
:10101000022010BD0D0C021110B50B460F22024923
:1010200001F06CFB10BD0000270C021110B50B463F
:101030000B22024901F062FB10BD0000370C0211C7
:10104000F72800D9F720084A01461080401EC31730
:101050009B0F18188003000C5080491EC80F4018C1
:10106000C003000C908070472851FF1F044A12886B
:10107000914203D8024A4000921D1152704700006D
:101080002851FF1F10B500231322194601F036FB2B
:1010900010BD000070B50C46880603D501F0F4FAC7
:1010A00020203AE0214D200409D5E878FEF7E4FF3E
:1010B000002801D0FEF7E6FF0120C0032DE0A007C5
:1010C0000026002805DA6E70012002F015FC0220CF
:1010D00023E020070ED504F073FF01F07DFA687855
:1010E000401CC0B26870062802D36E7001F0B0FBDD
:1010F000082012E0E00607D50D480078002801D14D
:1011000000F018F8102008E0E00708D00748083081
:1011100000F0FEF8FEF7BCFF0120604070BD6007E4
:1011200002D50420484070BD002070BDDC4EFF1F7A
:101130007C4FFF1F10B5024804F008FE10BD0000F0
:101140007927021110B50549054800F06DFB0348E9
:10115000044A0421083000F0E1FC10BDBC50FF1F20
:10116000FFFF0000907B021110B5034A0D210348D8
:1011700000F0D4FC10BD0000787B0211E44FFF1F8B
:1011800070B50E4C0025E0712572691EE18100F0FA
:1011900065FA04206072102200210948FEF77EFFE4
:1011A0000748102200211030FEF778FFE562E57055
:1011B000A57207202071E57270BD00007C4FFF1FF3
:1011C0000376FF1FFEB53B4D0C4608040CD5E879AD
:1011D000FEF752FF050004D002F06AF92846FEF738
:1011E00051FF0120C00360E0600403D501208003AB
:1011F0004840FEBD2F48E1070126007A00292AD089
:101200002978002920D0052821D0E9786846017086
:10121000A97A4170274906223031801CFEF71AFF57
:10122000297968460172E97A41726946E87900F0E5
:1012300001F9002808D007202872696A002903D024
:101240000968002900D0884720467040FEBD032071
:1012500069460870E4E7A1070DD5052809D1E8899A
:10126000FEF722FFAA8A002A03D00221E879FEF7BE
:1012700021FF022019E0600704D5002002F058F990
:10128000042012E0200712D5A879012802D00228F4
:101290000AD107E00096AB8B6A8B298BE88A00F0B5
:1012A0000BF801E000F050F808206040FEBD00207F
:1012B000FEBD00007C4FFF1FF8B5134C069E257A3B
:1012C000052D01D01420F8BD104F851FBD4219D245
:1012D000062917D3BD1DA94214D2FF27F537BA42FC
:1012E00010D20A2B0ED3AB420CD2E0822183628350
:1012F000A383304602F01CF90421E079FEF7E0FEFA
:101300000020F8BD1820F8BD7C4FFF1F7A0C0000AC
:101310001CB50B4C217A002901D011201CBD0028DE
:1013200000D06062064907482C31034601910090C5
:10133000103B0022617AE07900F016F800201CBD15
:101340007C4FFF1F1376FF1F10B50648017A052951
:1013500001D0122010BDC1891322C07900F0B4F968
:1013600010BD00007C4FFF1FF8B51D460224069FEC
:10137000079E0B00FEF7AAFE0D150815150815159A
:10138000151515151508150000F0B8F8040008D15A
:1013900032463946284600F067F900F0CBF801F0F4
:1013A00005F82046F8BD000070B5104C21680029F2
:1013B00004D00978814203D0032070BD122070BD93
:1013C0000B4D02212878FEF77BFE0A480026468056
:1013D00004212878FEF774FE074806802168032060
:1013E00048700020FEF778FE70BD00009451FF1F8A
:1013F000C551FF1FA851FF1F3851FF1F272803D2D7
:1014000002494000085A7047014870474051FF1F89
:10141000FFFF000010B5064C607004F067FC6078B8
:10142000FEF760FE0521607800F0BCFE10BD0000F4
:10143000C451FF1F70B5284E054630680C46002881
:1014400001D0112070BD254801780520014216D039
:1014500023488068002805D00078002802D0C807FB
:1014600006D101E0102070BD00F044F8002808D03B
:101470002078032805D0022803D0002801D01220AC
:1014800070BD0C20FEF734FE3060002820D00570BF
:10149000002141700A222146801CFEF7DBFD02F08C
:1014A0002BF9040002D001F033FB12E00D48007864
:1014B00003280ED11D20FFF7A1FF0B49002808804B
:1014C00007D00B48094A04210078FEF717FE00E018
:1014D0001324204670BD00009451FF1F3551FF1F9B
:1014E000A851FF1F3651FF1F3851FF1F60EA00004F
:1014F000C551FF1F10B504F017FC10BD70B50C46A8
:1015000005461C2200210948FEF7C8FD0848057061
:101510004470FEF7F9FD0549002803D0002008704B
:10152000122070BD01220A7070BD00005476FF1FAA
:101530003451FF1F70B50F4C0025A068002802D061
:10154000FEF7E8FDA560E068002802D0FEF7E2FDA6
:10155000E560094805210078084206D005481030AA
:1015600001F0A8FE01F076FA70BD002001F0A2FEA5
:10157000002070BDA851FF1F3551FF1FFEB5344D2F
:101580000C46080419D56878FEF776FD0121C903D9
:101590004C40064600280ED001F0ACFD002807D1D3
:1015A0002878FF2804D03146FEF7BAFD002802D083
:1015B0003046FEF767FD2046FEBDE0070127002804
:1015C0000AD0A868002804D04168002901D0002072
:1015D000884720467840FEBDA00709D568680028E6
:1015E00004D04168002901D00120884702202AE068
:1015F00060072AD5174E308800281FD0401E0004EF
:10160000000C30801ED101F0F5FA002809D01248F4
:1016100007706868002804D04168002901D00120C3
:10162000884701F0C1FA694600F01AFE684601F0E9
:101630004BFD1D20FFF7E2FE308003E004216878B7
:10164000FEF73EFD04206040FEBD0020FEBD000010
:10165000C451FF1F3851FF1F3751FF1F0149087048
:1016600070470000C451FF1F70B50E4C0B46261D7D
:1016700007C60546102200211846FEF757FD01282F
:1016800003D11021A06804F00DFF1022002128468C
:10169000FEF74CFD012803D11021606804F002FF21
:1016A00070BD00005476FF1F272807D2044A9142DC
:1016B00004D0044A400011520020704702207047B5
:1016C000FFFF00004051FF1FF8B50D4617461D49AA
:1016D00006461B4A1224C868954208D100282DD01E
:1016E0000268002A2AD029463046904723E0144A4F
:1016F000521C954213D1002807D00268002A04D05A
:10170000294630469047040005D03946304601F05E
:101710007BF9040012D10B48067047700EE0284692
:1017200004F0B4FA002809D00078B04205D1394657
:101730002846FEF701FD044600E003242046F8BDDC
:10174000FEFF00009851FF1FF8B50E4601461948EC
:101750001546007805221F46104028D0304326D079
:101760001548012E1BD0C468002C20D01F2D18D87E
:10177000002D01D0002F14D001701F220021601C09
:10178000FEF78CFC2A463946601CFEF763FC2846AF
:101790002570002E07D0611CFEF7D4FCF8BD8468CC
:1017A000E2E70220F8BD611CFEF7D2FCF8BD122072
:1017B000F8BD00003551FF1FA851FF1F014610B5AD
:1017C0000020C90704D0034A0421034800F0A6F909
:1017D00010BD0000C07A0211944EFF1F70B50F4D6E
:1017E0000F4CA87029461831204600F01DF8002142
:1017F00028460B461030CA0084521218491C0906AC
:101800005360090EF7D0012002F080FEA87800F0A6
:1018100023FB044804F0B0FA70BD0000744EFF1FB3
:10182000FFFF0000453D021170B50A4C0025A042A3
:1018300009D1002082008C525218401CC0B2957011
:101840000228F7D370BD02F04CFA0028FAD00480C9
:10185000857070BDFFFF0000F8B50E46074606997B
:1018600000240798002902D00B242046F8BD022B43
:1018700001D00D24F9E711785278120289188DB23F
:101880002946814301D08024EFE73846F16800F013
:101890003DF9A842E9D02A463846F16800F0A8F997
:1018A0000400E2D171892A46384600F065F9DCE788
:1018B00070B50C46080412D50A488078FEF7DCFBA8
:1018C000050008D02878B02802D1284602F026FB6F
:1018D0002846FEF7D7FB0120C003604070BD002002
:1018E00070BD0000744EFF1FFFB587B0087A002559
:1018F000109E1C460F46C0060DD5099802F0EAF965
:10190000030006D00A22394607989847050035D1CA
:1019100001E00E2532E0387802281DD178682922AE
:101920000178407812020002081880B2811A9042B1
:101930007ED009DC7249401A23D0012821D0022828
:1019400051D0032808D125E0012972D0022971D095
:1019500003296DD004296ED0099802F0E3F900281C
:10196000D7D00568002DD4D012991198019100901C
:101970003346224639460798A847054628460BB005
:10198000F0BD1198002873D1F86801783180027891
:10199000416897E0119800286AD101203080F868EA
:1019A0000021007820707889401C80B200F04EF948
:1019B00000280FD0318802788918891C3180817AFB
:1019C00061704189090AA17002784168E01CFEF744
:1019D00041FBD3E730880422001D30800021601CC9
:1019E000FEF75CFBCAE71198002872D1F86804A9D9
:1019F0000088009004203080009820700098000A31
:101A00006070009800F022F9070028D0F86805906F
:101A10006846028A03AB3B49384600F06FF900285C
:101A20000FD13B78022138487A68FFF70CF903E0C0
:101A300027E031E01DE049E0002802D13148694645
:101A400088810598007802280CD105980222416807
:101A5000201DFEF7FFFA3088801C308002E06946C6
:101A60000098888168468089A070000AE07085E748
:101A70002FE0119800282CD1F968079800F046F85B
:101A800004E01198002824D1F868008802213180F0
:101A90002070000A607071E7F868FEF75FFB11992B
:101AA000C0B2814210D8814201D1002206E0129AD0
:101AB0008918814202D31199401AC2B23280F96862
:101AC00011980918204682E7072557E71198002842
:101AD00001D00B2552E70721F86831800178217089
:101AE000417861708178A1704188090AE1700179BB
:101AF000217181796171C088000AA0713EE7000000
:101B000000280000FFFF0000127C021110B502F057
:101B1000E8F8002800D0807810BD00007CB514469D
:101B2000050019D068460195018000F09BF903007B
:101B30001DD1002C1BD06D89002D0DD00C20FEF77F
:101B4000D7FA00280AD0002303608580094A846000
:101B50009168002904D006E0022308E0132306E080
:101B6000906004E011460A68002AFBD1086018461C
:101B70007CBD0000744EFF1FF8B50C4C0746207862
:101B800015460E46FF280FD00A20FEF7EDFA010099
:101B90000AD0B12008700020487008714F80CE80B4
:101BA0000D812078FEF7BCFAF8BD0000744EFF1FCF
:101BB000FFB583B008461F4601A90C9E00F046F809
:101BC000050012D06846808802F0ACF800280AD0E0
:101BD0004468002C07D000963B462946059A039896
:101BE000A04707B0F0BD0E20FBE70120F9E7000099
:101BF00070B514460E46054602F073F8002806D16B
:101C00003146054802F06DF8002803D00580847045
:101C1000002070BD112070BDFFFF000010B50178DD
:101C2000B0290BD14178002908D10179122906D0B9
:101C30001B2903D14088012100F03EFA10BDFF218D
:101C40000231095C0129F5D010BD0000F0B58C46C9
:101C500010494B6819E09F687C89A04214D39E8884
:101C60003119814210D900220CE011017D186989D7
:101C7000814205D16046002800D004802846F0BD8E
:101C8000521C92B29642F0D81B68002BE3D1002080
:101C9000F0BD0000D051FF1FFFB5174881B00A9F6B
:101CA000446824E000251EE0A068290146187089D8
:101CB0000199884215D30299884212D804980028C5
:101CC00007D031787068049B039AFEF7BCFF0028A8
:101CD00007D0002F02D0A06840893880304605B078
:101CE000F0BD6D1CADB2A088A842DDD82468002CE0
:101CF000D8D10020F3E70000D051FF1FFEB51746F2
:101D000000256A469580044640891D4A1E46904239
:101D100008D001AA0092401C237880B26268FFF7C5
:101D2000BBFF05462378022116486268FEF78BFF49
:101D3000002807D12378022113486268FEF783FF49
:101D4000002801D060890EE0237802210F486268E4
:101D5000FEF779FF00280DD0002D03D0684680885B
:101D6000B84203D0384602F0CFFC04E06889401E38
:101D700080B200E06089002E00D030802846FEBD91
:101D8000FFFF0000107C0211127C0211167C021170
:101D900010B505490870042100F004FA00F006F8B7
:101DA000FEF7F0FF10BD0000E051FF1F70B50E4CB4
:101DB00000200C4B651CFF228100C91800280ED0A2
:101DC0000D80401CCA70C0B28A700228F4D3074844
:101DD00001F072FF064803F0CFFF002070BD0C80B9
:101DE000EFE70000D851FF1FFEFF00003946021147
:101DF000B9450211F8B50D4614460646694601F08C
:101E0000B7FD17280CD0002C06D001221021304637
:101E100003F016FF002803D129463046FEF7A8FF3D
:101E2000F8BD000070B50C46080411D509480078CB
:101E3000FEF722F9050007D00178A02901D101F0B1
:101E4000DFFE2846FEF71EF90120C003604070BD8A
:101E5000002070BDE051FF1F01490870704700006D
:101E6000D051FF1F70B50546008800281DD0686856
:101E70000221037842682248FEF7E5FE002808D1D7
:101E800068680221037842681E48FEF7DCFE0028DD
:101E90000BD01D4C6088002805D00122298812042F
:101EA000101A814203D9012070BD022070BD0C20A0
:101EB000FEF71EF9060001D000200AE0132070BDD5
:101EC00002016B6861880A329952491C401C61808A
:101ED00080B229888142F3D8002030600822294648
:101EE000301DFEF7B7F86068002802D1666004E094
:101EF000084601680029FBD10660002070BD000083
:101F0000107C0211127C0211D051FF1F0649496852
:101F100006E08A685289824201D188887047096840
:101F20000029F6D100207047D051FF1F10B51422B0
:101F3000114201D0012202E04A0604D500221021FC
:101F400003F07EFE10BDC80701D0002010BD0220A6
:101F500010BD10B514468A0604D50122102103F0E5
:101F60006FFE10BD882211420ED008220A401021B7
:101F700003F066FE00280BD0E034617E0029F0D02B
:101F8000217E0129EDD103E0880701D4032010BD93
:101F9000002010BD014610B50020C90704D0034A37
:101FA00007210348FFF7BAFD10BD0000AC7A02110B
:101FB000004EFF1F70B50D46164600241D49030054
:101FC000FEF784F808051234341934222934152D0B
:101FD00023D8162200211848FEF760F82A46314619
:101FE0001548FEF737F822E0022D16D11149108866
:101FF000103908801BE0082D0FD10E480822314609
:102000000838FEF7B7F812E0012D06D1CA69094970
:102010003078283107E0012D01D0182407E0CA6B81
:1020200004493078483102F036FC00E002242046B2
:1020300070BD0000004EFF1F2454FF1F0B7803707B
:102040000B8802221B0A43700B88801C012B02D0D4
:10205000022B07D011E08A7802704988090A417082
:1020600004220AE08A7802704A88120A42700A79C9
:1020700082708988090AC1700622104670470000E4
:1020800008B5044B009313460A46012103F028FDCE
:1020900008BD00003D2002111CB5032301920093EE
:1020A0000A46024B122103F04BFD1CBD01540211E4
:1020B00010B5FEF765F810BD13B504480078012887
:1020C00003D101AA6946FEF761F81CBDEC51FF1F60
:1020D00070B50F490F4A087000210B468C00491C4F
:1020E000C9B213530429F9D30A4C00211034FF2636
:1020F0000A460A256A4315196B80491CA354C9B2C4
:102100006E720329F4D3FEF747F803F0BDFC70BDEF
:10211000ED51FF1F7076FF1F082A01D00120704784
:102120004B780A781B02D2180280CB788A781B027F
:10213000D21842804B790A791B02D21882808A79A0
:10214000C97909025118C1800020704770B50C464A
:10215000080411D509480078FDF78EFF050007D067
:102160000178902901D103F0F1FB2846FDF78AFFA1
:102170000120C003604070BD002070BDED51FF1F05
:1021800070B500280AD1064C00252580A581A580C0
:10219000A068002802D0FEF705F8A56070BD000019
:1021A000FC76FF1F072907D0052905D0042903D095
:1021B000062901D002207047044A8B009A18134662
:1021C000403B1986203A9074002070477076FF1FBC
:1021D00070B506001BD10E4C0025214640310D7410
:1021E0004D740D76606D002802D0FDF7DBFF65654C
:1021F0005C20002546433419E80020184068002878
:1022000001D0FDF7CFFF6D1CEDB20A2DF4D370BDE8
:102210000C77FF1F70B50A880C460546072A07D0C1
:10222000052A05D0042A03D0062A01D0022070BD59
:10223000012103F0CFFD002804D02146284603F0F9
:10224000F5F870BD142070BD10B5001D80B2FDF70B
:10225000AFFF002803D00321C943FDF7AFFF10BD36
:1022600038B50C46050014D0002C12D00321684666
:1022700004F018F96946887840218006800E0843EA
:10228000694688702246284604F044FE050002D0C4
:1022900006E0022038BD03226946E01CFDF7DAFEA5
:1022A000284638BDF7B58EB00E9815460E46002864
:1022B0002DD0002D2BD0301DC0B20190FDF718FF9E
:1022C000040039D000F07CFC07463246201D0E99F0
:1022D000FDF77AFFF8B20890E0703804000E0B901A
:1022E000A0703802000E0A9060703F0E277000F058
:1022F00061FC0146102202A8FDF766FF06AB2146ED
:1023000002A8019A04F05CFD060003D010E0022050
:1023100011B0F0BD089828700B9868700A98A870E2
:10232000EF70082206A9281DFDF74EFF00F04EFCB5
:102330002046FDF7EFFE00E013263046E8E70000F8
:1023400010B5064C2070FDF745FF06212078FFF7F9
:1023500029FF034803F010FD10BD0000FC51FF1FD2
:10236000F964021170B50C46080419D50D480078BF
:10237000FDF782FE05000FD004F0DEF9002808D139
:1023800009480078FF2804D02946FDF7C9FE002837
:1023900002D02846FDF776FE0120C003604070BDE4
:1023A000002070BDFC51FF1FC451FF1F10B5054830
:1023B0000078400701D5044800E0002004F044FA0A
:1023C000002010BD3551FF1FF051FF1FFFB58DB02C
:1023D0000F98169C0E46002815D0002C13D00D988F
:1023E00003F054FC050011D06178207809024018F0
:1023F000A178E2780904120689184718286AB842B9
:1024000006D3401C04D0022011B0F0BD1420FBE71D
:10241000002E04D02879800701D40120F4E7082297
:10242000002106A8FDF73AFE1098001DC0B20190E9
:10243000FDF75EFE060017D0301D109A0F99FDF7CC
:10244000C3FE042221463046FDF7BEFE1022A91825
:1024500002A8FDF7B9FE06AB314602A8019A04F0C6
:10246000AFFC050002D013E01320CDE7082206A937
:1024700008A8FDF7A9FE0822211D08A8FDF7F6FD12
:10248000012801D0012503E039460D9801F08EF9AD
:102490003046FDF73FFE2846B6E700007CB5374CD6
:1024A000E07002F069FFFEF7FDF8FDF799FE0020ED
:1024B000009069460190FDF799FE032230493148AA
:1024C00005F0F2F92D25057002222F49401C05F078
:1024D000EBF9057002226946401C05F0E5F902217E
:1024E0001F20FFF7E1F803F0D5FE002001F004FA09
:1024F0002748284D0278254B01212878FFF724F939
:102500002648254B027800212878FFF71DF9244939
:102510000120214A08701078921C401EC1B2002090
:10252000FFF748FD7D20800103F0A0FE2021E07828
:10253000FDF762FE0025ED432846FFF72BFD2846F8
:10254000FFF73CF9FEF710FEFEF7FCFD00F02CF85B
:102550000120FDF757FE0120FDF75AFEF720FEF798
:102560006FFD0121E078FDF759FEE078FFF776F87E
:102570000C48FDF759FE00F06BF97CBDDC4EFF1FE7
:10258000E04DFF1F2376FF1FEC4EFF1FBE4FFF1FC6
:102590007D4FFF1F834FFF1FE475FF1F7E4FFF1FFF
:1025A000814FFF1F2257FF1F10B5094C07492046D6
:1025B000FFF73AF9054920460831FFF735F9034896
:1025C000044A07211030FFF7A9FA10BDF44EFF1F8F
:1025D000FFFF0000DC7A021110B5024803F0B6FBE1
:1025E00010BD0000D5780211002805DBC106C90E18
:1025F00001208840014908607047000000E100E0C8
:102600008307FF22DB0E9A408907090E99400028B4
:1026100008DB830809489B001B181868904308438F
:10262000186070470007000F0838830804489B00B3
:102630001B18D86990430843D861704700E400E054
:1026400000ED00E08307FF22DB0E9A408907090EA8
:102650009940002808DB830809489B001B1818686C
:1026600090430843186070470007000F083883083C
:1026700004489B001B18D86990430843D8617047F1
:1026800000E400E000ED00E010B5144800780028F8
:102690001BD0134C6078401CC0B26070C10715D0CD
:1026A00003F08EFC0F4800F005F90E491520FDF7E8
:1026B000C1FDA078002808D0401E0006000EA070C2
:1026C00003D17D20800103F02DFE10BD2428FCD312
:1026D0000020607000F0BCF810BD00007C4FFF1FB0
:1026E000DC4EFF1FBE4FFF1F10B5FDF7A9FD0120F7
:1026F000FDF7ACFDFDF7B0FD002010BDFFB583B0C8
:102700000F4603981B4940001646085AFFF79CFDE8
:1027100004002AD00125601C2670002F03D00699E2
:10272000B847401C85B2300610D51021039803F03D
:1027300051FB002801D0192613E06219E9B22046A6
:10274000FFF7B0FD06000CD10C35ADB20421684690
:1027500001800194058169460398FFF75BFD06003F
:1027600004D02046FDF71EFD00E01326304607B0DA
:10277000F0BD00002E51FF1F10B504460079BEB019
:10278000C00715D060880B49FFF7C0F9C0070FD00C
:10279000084800220830418D6846018001214180AF
:1027A0000548017A6846017160886946FFF722FB97
:1027B0003EB010BDBC50FF1FDE58FF1F10B5029C7D
:1027C0000020002C01D00B2010BD49680C784978FE
:1027D00009026118054C89B2A14205D10121198075
:1027E0000349097A117010BD0A2010BD192A000092
:1027F000DE58FF1F7CB515464A68069C167852784D
:102800001202B218104E92B2F24209D10122019284
:10281000DBB200942A46FFF71FF8040003D000E063
:102820000A2420467CBD69782878090240180749A7
:1028300080B209680029F4D0002802D0012088471E
:10284000EFE70220FBE70000FED6FFFFB850FF1FB6
:1028500010B502F0EBFC1120FDF704FD10490F4804
:1028600048631048016B012212051143016382681D
:1028700008210A438260826801231A4382600A4A5F
:102880001068FF231B0298430B0318431060074A8C
:10289000880610600648416310BD0000D54902114A
:1028A000C003FF1F40F000401CE400E000E100E036
:1028B0000000054030B5022202700123437006215A
:1028C000817016210171124D411C45710C462D0A73
:1028D00085714021C171002101720E490D78457248
:1028E00083720B7AC37202734A882273120A62736C
:1028F0000322C2738A880274120A42740C22827400
:10290000CA88C274120A02751121C17030BD00005C
:10291000D2FC0000DE58FF1F10B507480021C16639
:102920000920FDF7A5FC00210D2002F099F90021F6
:102930000C2002F095F910BD00500040F8B5496830
:1029400017460A784978069C090251182B4A89B221
:102950008A181E46042100250798091B1300FDF75D
:10296000B5FB06040D18242E3848042C33D28142BE
:1029700000D8084682B23280214835E0102C2AD295
:102980001021091B814200D8084682B232801D48BE
:102990002AE00F2C1FD20F21091B814200D80846C4
:1029A00082B21748328014301EE0042C13D28142C8
:1029B00000D8084682B212483280401D14E0042C30
:1029C00009D2814200D8084682B20D4832800A30CE
:1029D0000AE0042C01D307250EE0814200D8084606
:1029E00082B2074832800F3001193846FDF732FBBA
:1029F00002E0002030800A252846F8BDDCD5FFFF24
:102A0000547B02112376FF1F10B50C4603F052F9D8
:102A1000002804D040882146FDF78EFB10BD12200F
:102A200010BD0022002913D0002811D0012806D0A3
:102A30004A799206920E4A71032805D007E0487938
:102A4000C0221043487102E0402002434A71012233
:102A50001046704770B512480025007805210842DD
:102A60001BD02020FDF744FB0E4C0028A06013D0A3
:102A700020220021FDF712FB2020FDF739FBE0604A
:102A8000002804D020220021FDF708FB05E0A06803
:102A9000FDF740FB0020A0601325284670BD000014
:102AA0003551FF1FA851FF1F002909D0012807D168
:102AB000497989098901C02902D0402901D0022021
:102AC000704703207047FFB500200E4608701AE0DB
:102AD0001C5C401CC5B2002C17D02819904214D899
:102AE0005F5D6D1CEDB2384600F089FE002806D00F
:102AF000641EE0B2307000998F4202D1581904B0C0
:102B0000F0BD4019C0B29042E2D30020F7E70000C8
:102B100010B5044C2068002803D0FDF7FBFA002014
:102B2000206010BD9451FF1F70B50E4D84002859D0
:102B3000002815D0006A002801D0FDF7EBFA2859CB
:102B4000406A002801D0FDF7E5FA2859806A00287C
:102B500001D0FDF7DFFA2859FDF7DCFA00202851F3
:102B600070BD0000A051FF1F10B5044C6068002824
:102B700003D0FDF7CFFA0020606010BD9851FF1F11
:102B80000100044805D104498978002901D0024890
:102B9000801D70476476FF1F3451FF1F0148807805
:102BA000704700003451FF1F014840687047000023
:102BB0005476FF1F01488068704700005476FF1F5D
:102BC0000148C068006870475476FF1F10B5074879
:102BD000C0680168491C016005480078FF2803D0DF
:102BE00001218903FDF71AFB10BD00005476FF1F79
:102BF0003451FF1F02484068002800D00120704770
:102C00009051FF1FFFB581B00F460D9E0A9D03989E
:102C100003F03CF8040042D0019800283FD120790D
:102C20001021084320710499490702D50221084365
:102C300001E0FD21084020710B99284608430C99BA
:102C400008433043207902D00421084301E0FB21EE
:102C500008402071002E06D03069102220623146D3
:102C6000A018FDF7F7F9002D01D0002F05D00B9823
:102C7000002814D0012F08D011E0606A002801D08C
:102C8000FDF748FA1C21284606E0606A002801D0BA
:102C9000FDF740FA1C210B98FDF7F0FA60620398EB
:102CA000224C8700E05900283ED0002D0FD0006A4A
:102CB000002806D11C20FDF71BFAE1590028086204
:102CC00005D0E0591C22006A2946FDF7C3F90C988B
:102CD000002810D0E059406A002806D11620FDF7E0
:102CE00007FAE1590028486205D0E0591622406AE7
:102CF0000C99FDF7AFF9002E10D0E059806A00283A
:102D000006D11420FDF7F4F9E1590028886205D0B6
:102D1000E0591422806A3146FDF79CF90B9B049A16
:102D20000399019803F0A2F905B0F0BDA051FF1F6F
:102D3000F3B581B0019802F0A9FF050029D00E205B
:102D4000FDF712FA040024D02620FEF757FB0600F8
:102D500000D12E78D0202070002767700B20A07043
:102D60000622E91DE01CFDF775F9019860810298C3
:102D7000C1070120002901D0207300E027730299C8
:102D8000890701D5607300E06773F0B22146FDF753
:102D9000C7F9FEBD10B581881F4B0124CA1A99429C
:102DA00037D011DC1D4BCA1A994219D007DC1C4AD6
:102DB0008A1810D0022A1ED0032A29D11BE0472AE4
:102DC00027D0482A24D124E01300FDF77FF90621FB
:102DD0002222222222218068007800F0D1FC08E023
:102DE0008068827841781202891889B2007800F0F0
:102DF00027FD04460DE0094A921E914201D10122AD
:102E000000E0002280680178104600F001FD00E03B
:102E10000024204610BD0000532000000A200000BE
:102E2000FADFFFFF70B51A4D1A4A014600262878CE
:102E30001268194C01290CD0002A09D017490978C9
:102E4000490705D50221FDF73BF96680FFF760FED3
:102E500070BD6188002903D0114B1B78002B05D071
:102E6000002AF5D01078FEF79FFA70BD3C2902D3F6
:102E70003C39618070BD0221FDF722F962887D2016
:102E8000C000424302212878FDF714F9668070BD26
:102E9000C551FF1F9451FF1FA851FF1F3551FF1F40
:102EA0003751FF1F08B5418900910389C288818885
:102EB000C07800F0B1FB08BDF0B504468088A121C0
:102EC00089004843304987B009684018FF30FF3017
:102ED0000230A1794167002C54D02C4D686800283D
:102EE00023D006782A480068002804D041680029C9
:102EF00001D0002088472146E07908310591FFF78D
:102F0000D3FDE0710246277D638A218AE089019022
:102F100002A88AC0A0880090E0783146059B03F0A3
:102F20001BF9E078002802D00DE01A48D9E7E079D3
:102F3000E2896B46059907C3A379A188012230462F
:102F400002F052FEE0706868002811D0FFF70CFE16
:102F5000287800280CD06978FFF756FD002807D0A4
:102F6000E078A2880346297803F023F9002028702E
:102F7000A0881721FEF77AF8A088FFF701F9A0884A
:102F8000FFF726F907B0F0BD3409FF1F9851FF1F66
:102F9000C851FF1F3451FF1F70B5044600268088BA
:102FA00002F074FE002803D00678A08802F0F6FE36
:102FB000144D2878002808D0864206D16978FFF79A
:102FC00023FD002809D000202870002E05D0A37909
:102FD000A288A078314603F0ECF8A088094A810065
:102FE00008325158002901D0FFF79EFDA088172113
:102FF000FEF73CF8A088FFF7C3F8A088FFF7E8F8D1
:1030000070BD00009851FF1F70B58288294D0124C2
:10301000531B2949AA4242D019DC284D531BAA420E
:1030200018D00BDC264BD21826D0254B1033D218E3
:103030001ED0032A17D0042A39D10BE0012B09D066
:10304000022B07D0032B21D0042B30D11AE0433BB5
:10305000072B2CD8496800292AD00968002927D0D5
:103060008847044624E08068007800F0ADF81FE04F
:10307000806800F001F9F4E78068411C007800F0F6
:10308000D9F8EEE783681B78002B11D089680029F6
:103090000ED00B6808E0014610469847E1E7094961
:1030A0000968002904D04B68002BF4D100E000240B
:1030B000204670BD0E200000C451FF1F08200000F4
:1030C000F7EFFFFFA451FF1F10B5094CA1780029AD
:1030D0000CD001460622A01DFCF7BCFFA11DA07864
:1030E000FFF79FFCA01DFDF7CFF810BD002010BD1D
:1030F0003451FF1F1CB52F49037801240A68912B16
:1031000002D0A22B2ED13EE04178052909D00E290C
:1031100004D00F2908D03E2924D115E0FFF774FF11
:1031200010E0FFF739FF3AE001468088224B012486
:10313000C31801D0062B15D1002A30D05268002ABE
:103140002DD0904704462AE081780124032917D026
:1031500004DC012911D0022904D105E015291ED073
:1031600016291CD000241AE014498968002916D0B9
:103170004968002913D0884711E0FFF79DFE0EE053
:10318000FFF790FE0BE00E490978042909D0002AC8
:1031900005D05268002A02D001460A4890472046CE
:1031A0001CBD00216A46118001794088FEF768FF46
:1031B000F5E70000A451FF1FF3DFFFFFC451FF1F1D
:1031C0003551FF1FFFFF0000F8B5164F0646BD1F23
:1031D0002878FF2814D00A20FCF7C6FF04000FD07F
:1031E000D020207066700820A070A878E0700622B9
:1031F0003946201DFCF72EFF21462878FCF790FF6A
:10320000E87801280DD108480068002803D08068BC
:10321000002800D080470648044A04210078FCF7C3
:103220006DFFF8BD3A51FF1FC851FF1F60EA000053
:10323000C551FF1F70B500240546002805D100299F
:1032400003D006220B48FCF705FF0A481038017826
:10325000012907D10124002D06D000210170284644
:1032600000F0B6F9204670BD02210170FDF712F89A
:10327000F8E700006476FF1F10B50024002813D083
:1032800002780B49002A03D14288CA8202790A7661
:103290000A78022A08D102780124002A06D00022E6
:1032A0000A70007800F094F9204610BD0322F7E779
:1032B0005476FF1F0149486070470000C451FF1F4A
:1032C000F8B5794C8778014600250726E079227AFF
:1032D0003B00FCF7FBFE0805381C39396196CC38F9
:1032E000487800285ED1704806223C30C91CFCF7A3
:1032F000B1FE012020726278002A07D06A4B0121BA
:103300004233E079FEF720FA00284BD1A5E00F46C2
:103310004978002946D1F978002906D0634BA27874
:103320000021FEF711FA78700AE0022A0BD0012181
:10333000FCF7B6FF002803D10121E079FCF76EFF0E
:10334000787800282ED1F8BD497800292AD1032F9A
:1033500009D0A289002A0CD0217800290AD00121A5
:10336000FCF7A8FE06E0052A01D0022012E00620A4
:1033700010E02570207A062802D0042802D008E048
:10338000052007E0012020700146E079FCF746FFA8
:1033900063E00320207260E048780F46002803D0E5
:1033A00031282CD0267258E03F480622391D36308D
:1033B000FCF750FE7889E081B8892082F889608224
:1033C00005202072A28A002A03D00221E079FCF7AE
:1033D00071FEB889E083F8892084388A6084607936
:1033E00001280AD11F20FEF709F87D21C9004843B2
:1033F00002460421E079FCF75DFE25702DE0257082
:10340000C7E729480E46062200213630FCF746FE63
:10341000E583258465840421E079FCF751FE0821C9
:10342000E079FCF74DFEB07908280BD0032020721C
:10343000607800280ED02078002805D0E079FDF7CC
:10344000B3FF07E00420F2E7012020700146E07995
:10345000FCF7E4FE0020C043E081606A002800D150
:1034600071E701680029FBD0207A8847F8BD0D4636
:103470000821FCF725FE68780028F7D1E888E0836A
:1034800028892084688960840421E079FCF708FF9A
:103490000028EBD1A06A0028E8D00368628C218C58
:1034A000E08B9847F8BD00007C4FFF1FE475FF1FBD
:1034B00010B501781C4C912906D0A2291BD0D02927
:1034C00001D1FFF7FDFE10BD41780E29FBD18188A7
:1034D000164A9142F7D1816803200856217A0529BE
:1034E000F1D17F28EFD0616A0029ECD0496800292A
:1034F000E9D0884710BD41791329FBD10089012803
:1035000002D1A079022808D00520FDF777FF0246F6
:103510000821E079FCF7CEFD10BD0821E079FCF729
:10352000CFFDFDF711FF10BD7C4FFF1F05140000FC
:103530007CB5154C0546E08BE18A88420AD3218B85
:10354000884207D8208C618B884203D1608CA18B84
:10355000884217D00520FDF751FF0646E18A6846EC
:103560000180218B4180618B8180A18BC180E279B8
:103570006946E089FEF790FDA57132460821E079A1
:10358000FCF798FD7CBD00007C4FFF1FF8B5074697
:103590000E46084602F07AFB040018D02620FDF7FC
:1035A0002DFF050000D125780620FCF7DDFD040085
:1035B0000DD006220021FCF771FDD020207067702D
:1035C0000E20A070A680E8B22146FCF7A9FDF8BD48
:1035D00070B50F4D06462878FF2818D00E20FCF74E
:1035E000C3FD040013D0D020207066700020A070AE
:1035F00006220849E01CFCF72DFD06481038C18A58
:103600006181007E207321462878FCF789FD70BD1A
:103610003451FF1F6476FF1FFFB581B01E46174669
:103620000D460C20FCF7A0FD040013D0284602F044
:103630002DFB002810D00078D021217001996170F5
:103640000721A170A580E78026810A996181214622
:10365000FCF766FD05B0F0BD0048ECE73451FF1FF4
:1036600070B50D4D044628680E46002812D006207D
:10367000FCF77AFD010009D0D02008704C700320BF
:1036800088708E8028680078FCF74AFD002C01D0F5
:10369000FFF73EFA70BD00009451FF1FFFB581B0E7
:1036A0001F460E46084602F0F1FA050022D010200F
:1036B000FCF75AFD04001DD010220021FCF7EEFC9F
:1036C0002620FDF79BFE002800D12878D02121700C
:1036D000019961700F21A170A68003992172677210
:1036E0000A99A1720B99E1720C99E160C0B221466E
:1036F000FCF716FD05B0F0BDF0B51F4D85B028688C
:10370000002837D08778FDF7F5FE002805D00A207D
:10371000FDF774FE04900B200EE001F03FFE002840
:1037200005D00620FDF76AFE0490072004E008207B
:10373000FDF764FE04900920FDF760FE04460F4883
:103740000078002814D001262968C878091DFFF7E1
:1037500068F929686D46CA7A8B7A091D0BC50392F0
:1037600033463A4621460498FCF7A0FD05B0F0BD6B
:103770000026E9E70120F9E79451FF1F3651FF1FAA
:1037800010B50949096800290CD0002805D101208D
:103790004870FCF7A1FC002802D00021FFF760FF71
:1037A000012010BD002010BD9451FF1FF8B50C463C
:1037B00002F06CFA020021D026201462FDF71EFEF2
:1037C00005062D0E00D115789679D01D0090102099
:1037D000176AFCF7C9FC040010D0D020207000202C
:1037E00060700920A070E6700622201D0099FCF789
:1037F00031FC21462846E760FCF792FCF8BD411EEB
:10380000152903D9FF2801D00020704701207047F7
:1038100070B50A4E054630780C46FF280DD00420BE
:10382000FCF7A2FC010008D0D02008704C700220E8
:103830008870CD703078FCF773FC70BDA851FF1F05
:10384000F3B5284D81B0286800284AD04078264E2C
:10385000012803D03078002831D041E001F09EFDEE
:10386000224F002813D00120FDF7C8FD044641284F
:1038700008D91F4A02213878FCF740FC1D483C3C1F
:1038800044800EE07D20C0002246424303E0002039
:10389000FDF7B4FD0246002A03D002213878FCF778
:1038A00009FC2968022048703078002802D00020E6
:1038B000307015E002990198FFF7D2FE10E0032066
:1038C000019CFCF751FC010008D0D02008704C701E
:1038D0000420887028680078FCF722FCFFF718F9AC
:1038E0000120FEBD9451FF1F3751FF1FC551FF1F1F
:1038F00060EA0000A851FF1F10B5114902460B787D
:1039000008701048104900780978002B0AD0002A66
:1039100007D1022903D0062901D0042901D1FDF7DE
:1039200043FD10BD002AFCD0012905D0032903D096
:10393000052901D00429F4D10121FCF76FFC10BD49
:103940007C4FFF1F834FFF1F844FFF1F074A00213B
:103950008B00D35A834202D1880080187047491CDB
:10396000C9B20229F4D3002070470000D851FF1FCC
:1039700010B50C46FFF7EAFF00280DD0002C00D050
:1039800020608078FE2803D0FF2803D0162010BDC9
:10399000172010BD002010BD022010BDFFB581B062
:1039A000FF201E46174605300A9DFCF7DDFB04008C
:1039B0001BD0B02020706770029860802671002DA7
:1039C00006D02046FC2229460830FCF743FB05E0E0
:1039D0002046FC2200210830FCF760FB21460198BC
:1039E000FCF79EFB002005B0F0BD1320FBE70000B4
:1039F0000548172202800988172901D20420704740
:103A000001800020704700003051FF1F00207047E8
:103A100008B50A460888498888420BD8002809D08A
:103A2000002300931379521DFEF736F9002803D0C6
:103A3000002008BD012008BD0A2008BDF3B50D46D1
:103A400008884988002687B0814215D3002813D002
:103A5000002769460F710097002369881A46FEF710
:103A60001BF904004FD068460079002807D069464A
:103A70004979012925D008E0012009B0F0BD21785D
:103A800002291BD002216A4651711222504301AA19
:103A90006189801841806846007912235843801854
:103AA0001022001D6168FCF7D5FA68460079401CB9
:103AB0000106090E684601711FD11AE001216A460C
:103AC0005171217802291ED1820001A86189121842
:103AD00051806A4612796168920010180222001D16
:103AE000FCF7B8FA6A461079401CC0B2107105287C
:103AF00003D261890A48814200D101266089401CB5
:103B000080B2002EA7D068460079002805D001A910
:103B10000798FDF713F90020AFE70A20ADE7000092
:103B2000FFFF000038B50C4608884988884215D840
:103B3000002813D02379621D02210B48FDF783F87A
:103B400000280DD000200090237961882088621D14
:103B5000FEF7A2F8002805D0002038BD012038BDAE
:103B6000102038BD0A2038BD107C021108B50A4665
:103B70000888498888420BD8002809D00023009380
:103B80001379521DFEF788F8002803D0002008BDE5
:103B9000012008BD0A2008BDF8B500250F460646DD
:103BA0000C46E03717E06800205A0021FEF74EF877
:103BB000002809D0017A3046FEF7B8F9002808D06D
:103BC0006900615A2180F8BD6800205A20800120D8
:103BD000F8BD6D1CEDB2B87DA842E4D80020F8BD58
:103BE00010B5044608880021FEF730F8002804D0FC
:103BF000017A2046FEF79AF910BD012010BD0000A1
:103C000030B585B005466946FDF70CF9040026D1AC
:103C100068468078C1071E4809D08268002A04D00F
:103C2000688869469047044619E0062417E0426810
:103C3000002A05D0688869469047040001D10EE04B
:103C4000062468464078002809D1684681780173C7
:103C50000021C1810474688803A9FDF72FF8A868C2
:103C6000002801D0FCF79EFA002C05D16846807828
:103C7000122807D01B2803D068880121FEF71CFA00
:103C800005B030BD684640780128F5D1F8E700005E
:103C9000E051FF1F70B505460C4608880021FDF76E
:103CA000D5FF002805D0017A22462846FEF751F9B3
:103CB00070BD012070BD00000149486070470000E0
:103CC000E051FF1F10B50446801C00F029FDFF20C5
:103CD000E07010BD10B500F025F8002800D0806815
:103CE00010BD00229300CB5A834202D190004018AD
:103CF0007047521CD2B2022AF4D300207047000051
:103D0000074A0021CB00D35A834202D1C800801851
:103D10007047491C0906090EF4D0002070470000C6
:103D2000844EFF1F0649896805E08A88824201D1D6
:103D30008868704709680029F7D1002070470000A3
:103D4000744EFF1FF8B50746012906D0022924D179
:103D5000012102F03FF800281FD13846FFF7D0FFBD
:103D6000050015D000240D4E0CE0F8206968604372
:103D700008180188002908D0F8220021FCF78EF9E4
:103D8000641CE4B270788442EFD30020C0432880E2
:103D9000024938461831FDF747FDF8BD744EFF1F44
:103DA000F3B5064683B0083001900020009070887B
:103DB000FFF7A6FF07002FD0002523E0F820796841
:103DC00068430C182188002920D001980078012828
:103DD0000FD160880090A3887088A21DFDF7E8FECF
:103DE0000090002805D001990020087004982188CF
:103DF0000180F82200212046FCF750F900206D1CBC
:103E00002080EDB2074840788542D7D30020C043D8
:103E100038800098002802D17088FCF779FF00985C
:103E200005B0F0BD744EFF1FF3B50546374C06468E
:103E300085B00835F62200212046FCF72FF903A8AB
:103E400000902B79698828886A1DFDF725FF0746B1
:103E500045E070882E4A4100515C2E4BC91FC9B203
:103E60000093002202910192284B69468A89F63B11
:103E70003946FDF739FD002812D126482989001F4F
:103E8000828891420CD121492846F6390A30FCF744
:103E9000EDF8002804D02178788989000919488034
:103EA00068468289698804AB3846FDF727FF0746D4
:103EB0002078810009194A88002A10D0002F05D0E7
:103EC0006A46128A401C20708A800AE0020600219D
:103ED000920DC9431219401C2070918006E0002FFA
:103EE00004D00D48217800888142B2D32078002880
:103EF00006D070882146FCF713FF002007B0F0BD04
:103F00000698298801800A20F8E700002856FF1F3C
:103F10002E51FF1F784EFF1F2A51FF1FF0B585B0AD
:103F2000044600206946888120790E2869D00FDC7C
:103F3000082823D004DC022813D0062818D118E062
:103F400025460835484F0A281DD00C2810D138E0E6
:103F500010285BD012285ED0162861D0182877D19F
:103F600063E043484149008808806088FCF7B0FE60
:103F70006EE003A92046FFF757FF5AE003A9204649
:103F800000F076F955E0288804A9FDF75FFE0100EE
:103F900015D06088354E4200BA5C0023521ED2B262
:103FA0000193029200966A46B31C128AFDF79CFCAC
:103FB00000281DD160883146FDF738F848E001201F
:103FC00016E0288804A9FDF741FE0100F7D06088BB
:103FD0006B884200BA5C254E521ED2B20193029207
:103FE00000966A46B31C128AFDF77EFC002803D0B7
:103FF00029886A4691811CE060883146FCF7E6FF1B
:1040000026E003A9204600F0D3F912E003A92046D8
:1040100000F082F80DE003A9204600F039FA08E02C
:1040200003A9204600F028F803E003A92046FFF783
:10403000B7FE00280CD06178142909D00B492279E9
:104040000A706A4692894A8008716088FCF736FED9
:104050002046FDF7E3FD0748C168002901D020464E
:10406000884705B0F0BD00002E51FF1F2856FF1FE6
:104070002851FF1F744EFF1FF8B504460F46054632
:10408000083400896946FDF7E1FD06003AD0307A30
:1040900080060ED568460088FFF71CFE030006D098
:1040A0006888122231469847060002D02BE00E267F
:1040B00029E06E883046FFF723FE010005D1144841
:1040C000FFF71EFE01000ED00E80124A002052782B
:1040D00007E0F8264B6846439B5B002B05D0401C4D
:1040E000C0B29042F5D309260DE04968F82250434A
:1040F00008182146FBF7AEFF002668882146FCF72A
:104100005BFF02E00126208838803046F8BD0000C1
:10411000FFFF0000744EFF1FF3B58BB000200B9E15
:104120000746039004A800903246337B718930899A
:104130004C4C0D320836FDF7AFFD054678E00B9884
:10414000297A4088FDF7F2FE070003D00C986989B0
:1041500001806FE00B9844494088444B4200895CE1
:104160000093891FC9B20022029101923D4B69461A
:104170000A8AF63B2946FDF7B7FB0700E6D103980C
:10418000002833D039486188001F8088021D914281
:1041900053D1039909180B98408842003248805A3D
:1041A000801F814249DC0399A87A6118087103983D
:1041B0006989401C80B22218090A401C117180B222
:1041C00003906846028A718807AB2846FDF796FD82
:1041D000050011D003986946898B20180171039856
:1041E0006946401C898B80B2090A0CE01F48001FF9
:1041F0008088001D6080D6E70398FF212018017198
:104200000398401C80B222181171401C80B21749DB
:104210000390091F8A8813492018F639001DFBF7FF
:1042200019FF12490398091F8988401880B203902A
:10423000002D84D1039800280CD061880398FCF7E6
:104240003BF820700B9821464088FCF7C9FE0020FF
:104250000DB0F0BD002F00D10A270C9831880180E5
:104260003846F5E72856FF1F2E51FF1F784EFF1FD7
:10427000F3B50746044608378BB0494804903888A0
:1042800000252E4605906AE007A800903B797988C2
:104290007A1D0598FDF700FD0890002852D040894E
:1042A00005900898017A6088FDF740FE06005DD110
:1042B00060883C494200895C3B4B091FC9B20093AE
:1042C000002202910192364B69468A8BF63B08998F
:1042D000FDF70AFB060049D1002D36D0049841882D
:1042E0003148001F8088801C814241D12E4B1B1F0A
:1042F00098882918608842002A48805A001F814205
:1043000020DC0898817A04984019017108996D1C85
:104310004989E8B20A0A049909180A71401CC5B211
:10432000194604988A881E494019F639001DFBF782
:1043300091FE1D481D49001F00792818C5B2059837
:10434000884209D1002D13D123E017480499001F9A
:104350008088801C4880C9E7401C80B20590608836
:1043600041001048405A001FA8428DDA002D0ED09F
:10437000049841882846FBF79FFF01460498017086
:1043800060880499FCF73AFE00200DB0F0BD002EC5
:1043900000D10A260C99059808803046F5E7000000
:1043A0002856FF1F2E51FF1F784EFF1FFFFF0000F2
:1043B000F3B506460446002085B0324D009008361D
:1043C000288007463046E030049048E07800305AB4
:1043D00003A9FDF73BFC01001AD060882B4B8446F3
:1043E00042002948805C0093401EC0B20022029027
:1043F0000192244B68468289F63B6046FDF774FAC9
:104400000090002807D07800315A0698018035E0E6
:1044100001200090F7E71D492888091F8988421864
:1044200061884B001849C95A4B1E9A4204DD081A8C
:104430001649091F401E88802988A81C081813499E
:10444000091F8A880F49F639FBF704FE0F482988AF
:10445000001F8088081828807F1C0498FFB2807D88
:10446000B84207D96088298842000748805A401E10
:104470008142ABDB60882946FCF7CEFD009807B08F
:10448000F0BD00002856FF1F2E51FF1F784EFF1F62
:10449000F3B5054683B004460835008901A9FDF748
:1044A000D5FB2746E8370646002822D0307A80061A
:1044B0000ED568468088FFF70DFC030006D06088A3
:1044C000122231469847060002D013E00E2611E072
:1044D000002000906B88298860882A1DFDF768FB02
:1044E000060007D1787E002807D16088FCF7CAFD56
:1044F00003E00126049829880180787E002802D0F4
:10450000002005B0F0BD3046FBE70000F8B50446DA
:104510000246F820424319480025074645701037E7
:104520007868002807D00020C100C919401C000687
:104530004D60000EF8D0124E00213046FBF7AEFD64
:10454000002001466143C9B2F82251438B190B493F
:10455000C200103152180021536005E0F8274F4384
:104560005368491CDD53C9B2A142F7D3401C000671
:10457000000EE6D0014844700020F8BD744EFF1FC5
:104580003A54FF1F7CB50C78069D022C0FD14C6865
:104590002678647824023419064EA4B2F44206D177
:1045A0000224DBB200950194FDF756F97CBD012091
:1045B0007CBD0000FED6FFFFF8B505461D488542CC
:1045C00023D0461C002921D001292BD002291CD13F
:1045D0000121284601F0FEFB002816D12846FFF7EE
:1045E000B5F9040011D0A078FF280ED0FE2807D01E
:1045F00000200090E0781E2314222946FFF7CEF910
:104600002046FFF75FFBFF20A070F8BD2846FFF7AC
:104610009DF90028F9D13046FFF798F90028F4D029
:104620000580F8BD2846FFF791F90400F9D02680EF
:10463000D9E70000FEFF0000F3B50C468978C1B051
:104640001E2914D02E4D2878FF2829D0182927D8C4
:104650004808C2002B481218803A976F002F1FD0CD
:10466000D06F00281CD02078002817D113E0419883
:10467000FFF76CF905000BD000200090A378E878D4
:1046800000224199FFF78AF906462846FFF71AFBF0
:10469000304643B0F0BD6278012A03D1122901D01F
:1046A0000620F6E702AE0096A3886178A268B847B4
:1046B0000028EED1A0784008C100124808188038C0
:1046C000C26F02A94198904700280FD06178002955
:1046D000DFD1A27869460A70087168460189418075
:1046E00069464198FCF7EAFA0020D2E7A378042B48
:1046F000CFD00096002228784199FFF74FF9C8E7FC
:10470000D051FF1FAC7B021100B50346FDF7FEFB45
:10471000002803D0C018401E80B200BD184600BD5E
:1047200010B5040008D02078FF2805D0FE2803D05B
:10473000FBF7C8FDFF20207010BD0000F7B506464E
:104740000F461020FBF7D4FC05461020FBF7D0FCE9
:104750000446002D3AD0002C2DD010220021FBF76A
:104760009DFC2A462146304601F01AFE060023D160
:104770002878000604D43946284601F027FA08E0D4
:104780002146284601F022FA3A461149204603F014
:1047900031F93878000604D43846029901F016FA47
:1047A0000AE02146384601F011FA09492046029AEA
:1047B00003F020F900E013262846FBF7ABFC002CA1
:1047C00002D02046FBF7A6FC3046FEBD1326F6E7D6
:1047D000367C0211F8B5069800271D4614460E4691
:1047E000002801D00B20F8BD30780021022801D02C
:1047F00019804DE070680278407800021018152288
:1048000080B25202801A0300FBF760FC0504121FFD
:104810001A254100F068FBF7A1FCC2B2079882425A
:1048200000D902462A80F1682046FBF713FC30E0ED
:10483000F0680221008829802070000A607028E05A
:10484000062028800246F168EEE701202880F06803
:10485000007820701DE0F068002816D0082129801B
:10486000017821700188090A61708178A1704188FE
:10487000090AE170017921718188090A61718179E0
:10488000A171C088000AE07103E0298001E029805D
:1048900001273846F8BD10B50B78840702D50224ED
:1048A000234301E0FD2423400B7003070B7802D55E
:1048B0000824234301E0F72423400B7083060B7880
:1048C00002D52024234301E0DF2423400B700A217A
:1048D000084201D1810603D510780C21084304E079
:1048E000002803D11078F3210840107010BD00009B
:1048F000FFB581B0087800240A9E1F460D460228A5
:104900000FD168680178407800020818152180B23C
:104910004902401A09D0012829D0022848D003288A
:104920003CD00124204605B0F0BDE868FBF716FC3A
:10493000C0B2864205D8F0190090152803D90D247D
:10494000F0E70724EEE7E8683A4680190399FBF799
:1049500081FB0098EA6880B2002111541C4840682D
:104960000028DFD001680029DCD0002012E0002EF2
:1049700012D1022BE3D10399E8680A784978090239
:1049800051180180124840680028CBD001680029E6
:10499000C8D001208847C5E70B24C3E7002EFBD110
:1049A000062BCCD10622E8680399FBF753FBB9E745
:1049B000002EF1D1012BC2D103980078002803D03A
:1049C000012801D08024ADE7E9680870AAE700005B
:1049D000F04DFF1F70B5002530492E464D63304A1B
:1049E000284683009B189B68401C1B051B0D5D1906
:1049F0001E28F6D32B4888632B48066201202B49DA
:104A000040070860BFF34F8FBFF36F8F264C4034D1
:104A1000A06808218843A06025480078012803D0B9
:104A200060688902884360600021072000F05EF81A
:104A30000021072000F014F90021072000F042F9BE
:104A4000A06840084000A0601120FBF741FC112045
:104A5000FBF70EFC1120FBF7D3FA7720000145434A
:104A6000280C144C1449E080884214D27D2109019D
:104A7000884205D9401A0A21FBF730FC207200E079
:104A800026720E480078002804D10D4810210078C5
:104A9000FBF7C4FB70BD6420F0E700000000054098
:104AA00080050540FF01000000F0004080E100E0CB
:104AB0004A0AFF1FDE58FF1FB80B00007C4FFF1F84
:104AC000DF4EFF1F10B50448C16B034A4032106827
:104AD000D06000F0B1FA10BD0080004010B5002297
:104AE00011461120FBF700FC10BD000030B5C21FBD
:104AF0000A2A01D3062030BD162801D9052030BD71
:104B00000124074D9440002905D0002100F0DAF877
:104B10002868204301E02868A0432860002030BDB9
:104B200000380040162809D8054A01238340506800
:104B3000002901D0184300E09843506070470000FE
:104B400040380040162809D8054A01238340D06820
:104B5000002901D0184300E09843D060704700005E
:104B600000380040F3B50646FF2819D0B007C40E40
:104B7000B708651D304600F005FA0A48B900091863
:104B800088692B1B01225B1C9A40521EA240904355
:104B9000019AA2401043886101213046FFF7D2FFFD
:104BA000FCBD00000038004010B5114C20780028F2
:104BB00001D0072010BDFF2131310D48FBF79AFBD2
:104BC000012020700B490020086348630A490862ED
:104BD000486202211020FDF713FD1020FDF704FDAF
:104BE000064A07490D20FBF77FFB002010BD00009F
:104BF0005C52FF1F0080004080F00040494E0211CF
:104C0000B14D021110B5162801D9052010BD0C4B6D
:104C10009C6B01228240104620439863586B90435E
:104C20005863DC6B012907D020469043D863186B8A
:104C300002431A63002010BD10462043F6E700002F
:104C400000800040054B0122801E824058690029E7
:104C500001D0104300E09043586170470038004095
:104C600070B50D460446162801D9052070BD0021F7
:104C7000FFF768FF022C01D0032C03D1012120464D
:104C8000FFF7E0FF00212046FFF730FF0C4B01212A
:104C90001E190A460948A240012D09D041689143D6
:104CA000416002207070986990439861002070BD47
:104CB0004368134343607170F8E7000000800040D0
:104CC0005C52FF1F70B5162816D84200104B821890
:104CD0009E5CD218547893780E4D012213280CD282
:104CE000B0004519A868E41A641CA240521E9A40FC
:104CF000904399400843A86070BD6869E41A641C39
:104D0000A240521E9A40904399400843686170BD8A
:104D10002F7A021100F00040162801D901207047B7
:104D200007494A68012383401A4201D0096802E01A
:104D3000034940310969C140C807C00F70470000EE
:104D40000080004070B5162827D8184C4600164A37
:104D500035190123002912D014280BD0152809D0A9
:104D6000162807D0A0578000801881686A78934081
:104D7000194311E0506969788B40184312E01428F8
:104D80000CD015280AD0162808D0A057800080180B
:104D900081686A7893409943816070BD50696978F1
:104DA0008B409843506170BD00F00040747A02114E
:104DB000F8B50024124D01262F197878012808D162
:104DC0003146A869A140084216D0E0B20121FFF7A0
:104DD000B9FF787802280FD1E0B2FFF79DFF70404D
:104DE000E2B20146104600F07BF8E0B2FFF794FF14
:104DF0000C21614349194877641C172CDCDBF8BD92
:104E00005C52FF1F10B50F4C0D4A0123245C14287F
:104E100009D2106A002902D0A340184301E0A34040
:104E20009843106210BD506A002903D0203CA34073
:104E3000184302E0203CA3409843506210BD00009C
:104E400080F00040187A021170B502211020FDF7A1
:104E5000D7FB1020FDF7C8FB204D00242E197078D9
:104E600000281AD0022C01D0032C03D1E0B201217A
:104E7000FFF7E8FE707801280FD10121A869A14051
:104E800008420AD0E0B2FFF747FF0146E0B200F067
:104E900065F8E0B20021FFF755FF0C206043401990
:104EA000007F002816D0E0B200F090F8E6B2162E8F
:104EB00010D83046FFF730FF002801D0012100E074
:104EC00000210C2272435219527F824202D0304696
:104ED00000F0E6F8641C172CC0DB70BD5C52FF1FAD
:104EE000F8B516282ED842008318184AD55C9A18AF
:104EF0009278521ED4B2164A12185278022A21D140
:104F0000144EB76B0122134683401F43B763124B05
:104F100013280ED2002906D0A900C9188B68A24018
:104F200093438B600BE0A900C9188B68A240134320
:104F3000F7E70029596906D0A24091435961012140
:104F4000FFF760FFF8BDA2401143F7E72F7A021187
:104F50005C52FF1F0080004000F0004000B51628A2
:104F60000CD80123064A83400029116801D0194357
:104F700000E0994311600121FFF772FE00BD0000BF
:104F80000080004030B504460E48162C01D905209B
:104F900030BD0C210025614345540A4829461C3880
:104FA000001945702046FFF75BFE07494A6B012058
:104FB000A040824302434A630A6B82430A63284645
:104FC00030BD00007852FF1F0080004070B50446DD
:104FD00018480026162C01D9052070BD21460C2248
:104FE00051430D186A68002A02D1AA68002A1CD011
:104FF000104B02221C3B1B195A7001224254002103
:105000002046FFF72DFE6868002808D0A868002811
:105010000DD02046FFF780FE002808D0002631463C
:105020002046FFF7EFFD002070BD122070BD012665
:10503000F5E700007852FF1FF3B5184E002481B049
:10504000074601252846A040384223D0029908404F
:1050500000D001200090E0B2009900F021F80C206F
:10506000604380194168806800290ED0002807D06D
:105070000098002802D00021E0B203E00121FBE704
:10508000E0B20121FFF7BEFD04E0002802D0E0B24B
:105090000021F7E7641C172CD4DBFEBD7852FF1FFC
:1050A000084A16280DD80C2343439B185A68002A37
:1050B00001D0012904D09A68002A02D0002900D129
:1050C000104770477852FF1FF8B517460E46044642
:1050D0000A4DFFF757FF0C20604340198760466078
:1050E0002046FFF773FF050006490548086002D017
:1050F0002046FFF747FF2846F8BD00007852FF1F03
:10510000C54A0211C003FF1F10B50446162801D975
:10511000052010BD0121FFF7A3FD0548012102195B
:1051200051708269A1400A438261002010BD0000D5
:105130005C52FF1F30B58BB02C2217496846FBF735
:10514000DFF800246D46600041194978285CFFF7BC
:10515000B9FD641CE4B2162CF5D310484169C200B5
:1051600091430522120489184161416901225206C6
:1051700011434161416903225205914301225205C5
:10518000891841610120FBF7C1F8FBF7C5F8FBF76F
:10519000C9F80BB030BD0000E87A021100F0004001
:1051A0001CB51B491F2008701A48012404701A49B5
:1051B000002008701948C16B490949010931C163D0
:1051C000C16B602291432031C163FBF7B1F8FBF75B
:1051D000B5F800210420FDF735FA01211420FDF770
:1051E00031FA01211520FDF72DFA01211720FDF7D5
:1051F00029FA21030A48FBF7A7F803200346009089
:105200000122084901940848FBF7A4F81CBD0000DE
:10521000480AFF1F490AFF1F680AFF1F80F000406D
:10522000E465FF1FE858FF1F6063FF1F70B5294D3D
:1052300000202862274C4034A06840084000A0604D
:10524000A06808218843A0601120FBF711F8112005
:10525000FBF73EF81120FBF783F8E86B4021084389
:10526000E8632068090308432060606880210843E0
:105270006060606889038843606060680912084361
:105280006060E06B10218843E063E06B012108431C
:10529000E06308022862E16A0F480140E162216B85
:1052A00001402163616B01406163A16B0140A16317
:1052B000A0680121C9058843A06000210720FFF7ED
:1052C00001FD01210720FFF72DFC01210720FFF739
:1052D0000DFC70BD00F00040EFFFEFFF70B5002146
:1052E0000D20FFF73FFC01210C20FFF73BFCFBF7F3
:1052F0003DF805461A4C0920FBF732F80021E1661B
:1053000061202060206806229043001D206015481F
:10531000854203D10A20E06111201AE0124885423B
:1053200003D11E20E061232013E01048854203D101
:105330003020E06136200CE00D48854203D1432047
:10534000E0614B2005E00B48854203D16920E06114
:10535000712020622163A1630120E06370BD000021
:10536000005000400024F4000048E801006CDC021A
:105370000090D00300D8B80510B5064A06490420AD
:10538000FFF7A2FE1120FFF7BFFE01211120FFF75A
:10539000E5FD10BD615E0211315F021108B50948DB
:1053A0008368002B0CD01A78694601205B1CFDF73E
:1053B0008AFB002804D00078C00701D0012008BD76
:1053C000002008BDA851FF1F10B503460B4A00205E
:1053D0000A21414389184988002905D0401CC0B2E0
:1053E0000328F5D3002010BD0A2100244143545462
:1053F0000446403488184480037210BD8076FF1F35
:105400000A7802700A88120A42708A7882704A8882
:10541000120AC2700A7902718A88120A42718A7964
:105420008271C988090AC17108207047F8B505461C
:105430000C4648680421FAF7C1FE217A01702189DF
:105440000346401C090A0170217841702188090A2D
:105450008170207A001DC2B2FB2A36D81C488542D2
:1054600015D114461E460C20FAF77EFE01000CD022
:1054700090200870022008714D808E601548CC8005
:105480000078FAF74DFE00271DE013271BE05C2093
:1054900011496843441826464036307E002806D01D
:1054A00008465C30416A0727491C41620BE02146EF
:1054B000284600F095F90746307E002803D12146A2
:1054C0002846FBF7AEF83846F8BD0220F8BD0000CC
:1054D000FEFF0000ED51FF1F0C77FF1F10B50A4AB9
:1054E00000210A234B439B185C88002C06D01B79B3
:1054F000834203D10A204143881810BD491CC9B218
:105500000329EED3002010BD8076FF1F00214180CB
:105510000170704770477CB504000FD06088002888
:105520000CD00025009501951323E188207A1722DD
:1055300000F028F8FF206072658025707CBDF8B50A
:10554000074615460E461020FAF70EFE040017D047
:10555000A0202070002060706680002D05D00C22F5
:105560002946201DFAF776FD04E00C220021201DBB
:10557000FAF794FD21463846FAF7D2FD0020F8BD2F
:105580000120F8BDFFB581B01E46174614200B9DC3
:10559000FAF7EAFD04001AD0A22020706770029882
:1055A00060800A9820716671002D06D020460C227A
:1055B00029460830FAF74EFD05E020460C2200216E
:1055C0000830FAF76BFD21460198FAF7A9FD05B0FE
:1055D000F0BD022A1CD34B780A781B02D21892B273
:1055E0000280012A02D0022A06D00FE08A78C97808
:1055F00009025118418009E0CB788A781B02D21841
:1056000042800A7949790902511881800020704747
:1056100001207047F8B506464D88002070600A7971
:105620000C46022A12D0290160480091415A0029F3
:1056300006D0009B1F18BB68002B01D0012A7DD02B
:105640005A486C304169491C4161A9E0E288042A4A
:1056500043D3A068437801781B02C91889B200912E
:10566000C37881781B02C9188FB2017AC079000211
:1056700008184F4948800099091D8A4220D1072FF8
:1056800013D0052F11D0042F02D0062F25D10CE006
:1056900046482901405A002807D02846FCF770FDEB
:1056A00042486C300169491C0161009830813780A3
:1056B0000321C943A068FAF781FD70600020F8BD9E
:1056C000072F18D0052F16D0042F07D0062F12D081
:1056D00036486C30C168491CC16064E03348290118
:1056E000405A002807D02846FCF74AFD2F486C3066
:1056F0000169491C01612D492D01002048536E1894
:105700000098B081B7800098FCF79EFDB06000283B
:1057100018D00321C943A068FAF750FDE28801467A
:10572000224F121FB068FAF795FC785BE1884018A9
:10573000001F785338466C30016800E008E0491CCF
:10574000016030E019486C308169491C81612AE0B0
:10575000E2888918009A89B28152BA8991421AD88E
:105760000546B868E2884018801AA168FAF772FC0A
:105770000098295AB889814215D13081B888308083
:10578000B868706000990020685208486C30416821
:10579000491C416007E005486C308168491C816004
:1057A0002846FCF7EDFC0120F8BD0000FC76FF1F49
:1057B0000652FF1F022A01D0012070470A7849785B
:1057C000090251180180002070470A7802704A7857
:1057D00042708A78C97809025118418070470000E8
:1057E000FFB50C4607463D49A12080000968784373
:1057F0004018FF30C130067E89B015463846FBF7A9
:10580000B1FA001DB04204D23846FBF7ABFA001DD6
:10581000C6B2B54207D82A46002138460C9BFAF793
:10582000EDFE0DB0F0BD31462846FAF745FD27469E
:10583000403738740C99616501467143691AC9B2E1
:1058400002910C9904910299002901D0401C3874EE
:10585000002523E00299002904D0401EA84201D16E
:10586000084600E03046E900059103916054FCF7DA
:105870001FFC03990919486000281BD00599625C38
:105880000499FAF7E7FB0598215C0498081804903E
:105890001348C169491C6D1CEDB2C161387CA84236
:1058A000D8D8606D002803D0FAF77CFC0020606532
:1058B0000020B6E7002038740646606506E0F00078
:1058C00000194068FAF76EFC761CF6B2AE42F6D3C9
:1058D0000348C16A491CC1621320A2E73409FF1FB3
:1058E0006877FF1FF7B586B016460D464878FFF774
:1058F000F5FD040010D0002727712878012802D078
:10590000132809D105E06A88314602A8FFF761FE35
:105910000AE02078032802D0002009B0F0BD6A8890
:10592000314602A8FFF746FF0646204600F046F93A
:1059300002A8019000972B78207A32460699FFF74B
:1059400021FE2046FFF7E2FD3046E6E7FEB50446BD
:10595000468801466846FFF75DFE05460198002827
:105960002FD068460088052806D0042809D00628CC
:1059700007D0072805D026E06946304600F030F809
:1059800021E081001548081801464039098E002998
:1059900019D02038807C6A463146FFF7D0FD0028B8
:1059A00011D168460088042803D001213046FCF755
:1059B00083FB012D04D1A068002801D0FAF7F2FB87
:1059C000FEBD012D04D1A068002801D0FAF7EAFB42
:1059D00001213046FCF770FBFEBD00007076FF1F12
:1059E00030B50546088987B00C46042817D302A8AD
:1059F0006168FFF7EAFE68464089172837D8218991
:105A0000001D81421ED16846007AC10709D0626834
:105A100002A92846121DFFF765FF002812D107B022
:105A200030BD6168091D122805D000206946088034
:105A3000497A6A4622E06846428903A8FCF76CFB73
:105A4000002803D02846FFF765FDE8E70D48818868
:105A50000029E4D06946497A03AA01920091694677
:105A60000B7A807900222946FFF78CFDD7E70121C8
:105A70006846018017214180417A6A462846FCF732
:105A8000FFFACCE77076FF1F70B5144C0026268015
:105A9000A681A680A0683546002802D0FAF782FBCE
:105AA000A5600E4C103420464030057445740576D0
:105AB000606D002802D0FAF775FB65655C20002553
:105AC00046433419E80020184068002801D0FAF74E
:105AD00069FB6D1C0A2DF5DB70BD0000FC76FF1F15
:105AE000FFB589B015460E461720129FFCF7ACFB98
:105AF000040021D0684606704570002F03D0201D99
:105B00000C99B84700E0002069464880267065700F
:105B10004888A070010AE170052269468A82001D4A
:105B20000694888305A90998FFF780FC050004D036
:105B30002046FAF737FB00E0132528460DB0F0BDEC
:105B4000FFB581B01E46054601210A9F0B9C00F05F
:105B500041F9002811D02046FFF736FC00280AD072
:105B6000C5800446077012484178491C0A06120E87
:105B7000427004D005E015250FE014250DE0012248
:105B80004270227100962846039B0299FFF7A8FFF6
:105B9000050005D02046FFF7B9FC284605B0F0BD4A
:105BA00023462146034A09330348FAF7E5FBF4E7A5
:105BB0000652FF1F307500001755021110B504463C
:105BC000407AFAF77FFBFF20607210BD10B5002409
:105BD0000F22835C5B0023438B54835C521EDC09E1
:105BE00052B2002AF5DA10BDFFB581B01E46174645
:105BF0000D46084600F04AF8002802D0112005B0F2
:105C0000F0BD0E4800F042F8040015D00A98A071CB
:105C10000622E01D0B99FAF71DFA6580277166715F
:105C200001982070002060620C98E08100212846D5
:105C300000F008FA0020E2E71520E0E7FFFF00008F
:105C400070B514460D46064600F020F800280BD02B
:105C5000416A007900290CD0C20611D580070AD408
:105C6000002C08D0052070BD074886420AD01420B9
:105C700070BDC006F6D5887EA84203D20C2070BD48
:105C80000F2070BD002070BDFEFF0000084A0021FB
:105C900028234B439B185B88834203D12820414330
:105CA00088187047491C0906090EF1D0002070477A
:105CB000A076FF1F30B50B4C0B4B002128224A4326
:105CC000D5186D88A54206D09A5C824203D128205F
:105CD0004143C81830BD491C0906090EEED000200A
:105CE00030BD0000FFFF0000A076FF1F10B50020B0
:105CF0000B4C0C4B014628224243D2185480401CC6
:105D0000117100065162000EF5D0064A00202832BB
:105D10008300401CC0B2D1500528F9D310BD00004B
:105D2000FFFF0000A076FF1F0020074A014628233E
:105D30004B439B181B79002B01D0401CC0B2491C5F
:105D40000906090EF3D07047A076FF1FF8B50500CD
:105D50000DD0074F074E002428206043801941884A
:105D6000B94200D0A847641C2406240EF4D0F8BD24
:105D7000FFFF0000A076FF1F074A00218B00D358C9
:105D8000002B05D0491CC9B20529F7D31320704751
:105D90008900505000207047C876FF1F10B5FFF7EC
:105DA00075FF040013D06088012100F04BF9606A90
:105DB000002801D0FAF7AEF9282200212046FAF790
:105DC0006DF90020C04360800020207110BD0220CA
:105DD00010BD000010B50C460649884206D0FFF7FA
:105DE00055FF002804D00079204201D0012010BDC9
:105DF000002010BDFEFF000070B5154C0220207081
:105E0000144D012028700020FAF7BCFAFAF7C0FA06
:105E1000FAF766FCFAF7C2FAFFF7C2F9FFF78AF958
:105E20002078FAF7C1FA2878FAF7C4FAFAF7C8FA2C
:105E300009490420FAF7CAFAFEF7B6FE022107481C
:105E4000FAF7CAFAFEF74AFEFCF74EFC002070BDD6
:105E50004A0AFF1F744FFF1F3B00010800C00311D7
:105E600010B5002902D11120FFF778F810BD00000D
:105E700070B500241420FAF73BF916491422086083
:105E80000021FAF70BF920460124FAF7ABFA0225B4
:105E90002046FAF7ADFA2846FAF7B0FA03200425AF
:105EA000FCF716F905242846FCF74AFA0625204691
:105EB000FBF7B0FA07242846FBF76AFF08252046BF
:105EC000FBF75EF909242846FBF788FC2046FCF71F
:105ED000E5FA70BD784FFF1F70B50546114C0026DE
:105EE000E0782B00FAF7F2F8061C0408171C0D1CCA
:105EF0000221FAF793F913E00821FAF7E1F8667046
:105F00000EE0A670084A0821FAF7F8F80021E078B8
:105F1000FAF77AFA04E00121A1700821FAF7D0F823
:105F2000257070BDDC4EFF1F102700007047000079
:105F300010B501290DD107491320887001211120C6
:105F4000FFF70CF804480078002802D0034800F05E
:105F5000E9F910BDDC4EFF1F7C4FFF1FC409000094
:105F6000FFB5154C81B000211D4617461E46E1665F
:105F70006060FAF74FFA0120E06602982061A015F0
:105F800000E02061761EFCD2FAF74AFA0B4801685D
:105F90000DE0226F120703D522693A706D1E7F1C37
:105FA0000268521A0A2A02D9012005B0F0BD002D5C
:105FB000EFD10020F9E70000005000406008FF1F0B
:105FC00038B5FFF78BF902236A4600214020FFF71E
:105FD000C7FF044600AA0223012140200232FFF736
:105FE000BFFF0443FCF798FC002C03D0FAF75AFBE0
:105FF000012038BD694608880D4940BA00B20D4AF3
:106000004843801801140C480C4B4180694649886C
:1060100049BA1140594389180914094A81809142AB
:1060200000DD82800188491C0180002038BD00000D
:1060300006640000FF7F0000DE58FF1F204E0000B6
:106040000F270000F8B5084D0E4607460024A000B3
:106050002A58002A02D0314638469047641CE4B2E0
:10606000052CF4D3F8BD0000C876FF1FFFB581B042
:106070000298FFF70BFE040069D0029835498600AC
:106080008A59002A63D0136A1820002B00D03420CC
:10609000936A002B00D01430049B002B00D01C30DE
:1060A000516A002900D01630FAF75EF805004ED08C
:1060B00018220021F9F7F2FF2620FBF79FF90700CD
:1060C00000D12778D0202870019868700A20A87025
:1060D0000298A8800398A8711E482C46805918344D
:1060E000006A002808D01B49AC60895920461C343E
:1060F000096A1C22F9F7AEFF16488059806A002809
:1061000008D01449EC60895920461434896A142255
:10611000F9F7A0FF0498002806D02C6120461C3413
:106120001C220499F9F796FF0A488159496A002907
:1061300006D06C6180591622416A2046F9F78AFF21
:10614000F8B22946F9F7ECFF0298FCF7EDFC05B030
:10615000F0BD0000A051FF1FFFB581B01D461746DE
:1061600014200E9EFAF700F8040020D0D0202070F2
:10617000019860700520A070E770002D05D0062200
:106180002946201DF9F766FF04E006220021201DA4
:10619000F9F784FF0A9860810B98A0810C98E08140
:1061A0000D982082A67421460298F9F7B9FF05B030
:1061B000F0BDF8B506461C4615460F460820F9F70F
:1061C000D3FF010009D0D02008704E7006208870DF
:1061D0008D808C713846F9F7A3FFF8BD70B50D4678
:1061E0000B4C0021E1666060FAF714F90120E066CB
:1061F0002561FAF715F907490868626B920505D41D
:106200000A68121A0A2AF8D9012070BD002070BD50
:10621000005000406008FF1F70B50E46114C002171
:106220001546E1666060FAF7F5F80120E066266140
:10623000606BC006FCD5280A2061606BC006FCD5E7
:10624000E8B22061FAF7ECF807490868626B92053A
:1062500005D40A68121A0A2AF8D9012070BD002054
:1062600070BD0000005000406008FF1F10B50446DC
:1062700001460620FBF718FA21460720FBF714FA1F
:1062800021460820FBF710FA21460920FBF70CFAFB
:1062900010BD000038B51E48FAF7C8F8022817D01C
:1062A0001C4C6B4606221A492046FAF7C5F800280E
:1062B0000ED003211648FAF7C5F815498D20C8708D
:1062C0001F2008713820487106222046FAF7C0F8CE
:1062D00012490D200870104C0C20207009206070AD
:1062E000A41C0B4D04220E492046F9F7B3FE241DD1
:1062F0002D212170601C0122A91C01F0D5FA012278
:10630000691C01F0D1FA0122294601F0CDFA38BD0D
:106310006509FF1FADAC0000E475FF1F7E4FFF1F36
:10632000547B021110B5FFF7A1FF064C2078FBF754
:106330003BF805490420087001212078F9F76EFF29
:1063400010BD0000834FFF1F844FFF1F00784107DF
:106350008207C90F920F89000006C00E1143C000CA
:106360000843704701468A000849102089580029CF
:106370000AD00A6A002A07D08968002904D0107A56
:10638000097E884200D30846704700001052FF1F64
:1063900010B50246014620321031FAF75FF810BD01
:1063A00010B5FAF75BF810BD7FB50D4604468100C5
:1063B0000948405800280ED0014668314EC903965E
:1063C0006E460EC6037FC28801782846FCF71AFC89
:1063D000204600F003F87FBD1052FF1F70B5044641
:1063E00000F0BEFCA500134C6059002821D0006AC3
:1063F000002801D0F9F78EFE6059806E002801D088
:10640000F9F788FE6059C06E002801D0F9F782FEC6
:106410006059006F002801D0F9F77CFE6059406F89
:10642000002801D0F9F776FE6059F9F773FE0020D5
:10643000605170BD1052FF1F7FB5084D840029596F
:10644000102268462531F9F705FE2859044BC0880B
:106450006A46112100F014FC04B070BD1052FF1FF9
:10646000A57102117FB50C4C85006159002910D02F
:10647000694600F029FC60590178C088002901D0E4
:10648000064B00E0064B6A46072100F0F9FB04B01A
:1064900070BD0120FBE700001052FF1F01720211C6
:1064A0009372021170B50D46064600240AE0F9F712
:1064B000DBFF010A3155641CE4B2AC4202D2305514
:1064C000641CE4B2AC42F2D370BD00007FB5084D4D
:1064D00084002959102268463531F9F7BBFD285947
:1064E000044BC0886A46112100F0CAFB04B070BD9D
:1064F0001052FF1FDF71021110B5064A8300D258F7
:10650000002A06D0D288824203D1012901D1FFF7A7
:1065100065FF10BD1052FF1F70B50E4C064685007A
:106520006059002813D000782146002810D08868D0
:10653000002804D04168002901D0304688476059BE
:106540004078122803D100213046FFF72DFF70BD9F
:106550004868EDE71052FF1F10B50A46024B1121A3
:1065600000F08EFB10BD00000D7102111CB5044639
:1065700068461346017006221946401CF9F76AFD69
:10658000034B6A460821204600F07AFB1CBD000040
:106590002F71021110B50A46024B112100F070FB59
:1065A00010BD00005571021110B586B00446684652
:1065B0001346018008221946801CF9F74BFD044B55
:1065C0006A460B21204600F05BFB06B010BD0000C0
:1065D0007771021110B50A46024B112100F050FBF1
:1065E00010BD0000A172021130B587B00446002032
:1065F00069460875A06805782B00F9F767FD0C2C33
:1066000007070F1215181B1E2124272C00F0CAFEA5
:1066100012281DD106206946087529E000F094FE75
:1066200016E000F0B0FE13E000F09DFE10E000F078
:1066300048FE0DE000F074FE0AE000F062FE07E0A4
:1066400000F04EFE04E000F025FF01E000F014FF32
:10665000002802D008E00720DEE760886A46294665
:1066600000F028FF694608756846007D002805D0BF
:10667000608805A900F0F2FA07B030BD608800F02C
:1066800043FBF9E7F8B52B4D06468700E8590C4661
:10669000002807D0C188B14204D14178062904D02E
:1066A000112930D0002C36D03EE002782149002A52
:1066B00025D08368026A5B69DC0704D0147BE40799
:1066C00001D0072105E09C0705D5147BA40702D55E
:1066D000092141702CE05B0704D5127B520701D5DC
:1066E0000B21F6E78868002822D0416800291FD0D6
:1066F00030468847E8594078122802D018E04868A8
:10670000F1E7002103E0002C00D03224214630467E
:10671000FFF74AFE0CE03046FFF7B8FA002803D036
:10672000017910221143017131462046FCF72EFFFA
:106730000120F8BD1052FF1F70B501780124922985
:1067400002D0A02919D130E041780E2902D03E298B
:1067500013D10BE081881A4AD14205D18068411CCF
:10676000007800F033F81EE000201CE0014680783D
:106770000124052803D0082811D000241DE0114869
:106780000078400719D510480068002815D08368A4
:10679000002B12D0CA898888891D984703E0888811
:1067A0008979FFF76FFF044607E00546FFF71CFFF6
:1067B000A868002801D0F9F7F5FC204670BD00005C
:1067C000E8DFFFFF3551FF1F1452FF1F70B51D4C4E
:1067D00005462068002825D0002D06D10278002A21
:1067E00021D008220A30F9F735FC20682E4600280F
:1067F00017D01220F9F7B8FC05000DD0C120287081
:106800006E7021681022A81C891CF9F723FC2068EF
:1068100029464078F9F784FC2068F9F77BFC0020D2
:106820002060012070BD0822801CF9F713FCF9F7E5
:1068300021FE002801D00125D7E72168012008703A
:10684000EFE700000C52FF1F01494860704700004D
:106850001052FF1FF7B588B01646044610220021DB
:106860006846F9F71BFC334DA700E859002835D0DE
:10687000C188A14232D1017800292FD14278062A5D
:106880000FD0816E002929D0088A112A19D0B04270
:1068900024D1082212310998F9F7E8FB01283CD0ED
:1068A0001CE0024601465532353104AB0C3000F095
:1068B00000FC002812D12046FFF754FD024604A92F
:1068C00030E0B04206D1082212310998F9F7CEFB28
:1068D00001281BD032212046FFF766FD2046FFF736
:1068E000D5F905000CD0696A002909D0088AB042A0
:1068F00006D1082212310998F9F7B8FB01280FD008
:106900002046F9F7BDFD01200BB0F0BD2046FFF792
:1069100029FDE9590246896E04E0E859816E00E0DC
:10692000696A8A7E6846F9F795FB20466946F9F759
:10693000ADFDE8E71052FF1FF1B582B00298694C37
:10694000850060590178002976D141788768066A08
:10695000062907D0CA1F1300F9F7B8FB050A4852E9
:106960005B1872007969CA0706D0327BD20703D060
:10697000806E002813D019E0880702D5307B80078D
:106980003ED4480764D5307B400761D5FCF712F947
:106990006159CA8801461046FFF71CFE58E01C20CA
:1069A000F9F7A6FB61590028886653D06059102278
:1069B000866E00213046F9F771FB0298FFF7D2FC92
:1069C00001463046FFF76EFDF9F74EFD3082304646
:1069D00008211230FFF766FD0298FFF7C3FCB0767E
:1069E00060593146C088FFF7B7FD33E0816E00295A
:1069F00032D00A461232098AC088FFF7D5FD2BE053
:106A0000FCF7D2F86159CA8801461046FFF7C2FD6B
:106A10003FE001200190FCF7C1F8009001280CD064
:106A2000002000900198FCF7ABF8024660590099ED
:106A3000C088FFF79BFD39E023E000200190F2E7DA
:106A4000072907D0082907D0092922D00A292DD0E3
:106A500078690EE008201DE07869810704D5317B54
:106A6000890701D5092015E0410721D401E00B2059
:106A700010E0C10520D5B189C9051DD50C2061598B
:106A80004870FEBD40051ED5B08940051BD51020BD
:106A9000F5E70A20615948706059C088FFF7F6F899
:106AA000002812D0C08941080A1810E07869DBE795
:106AB000317B4907DDD5DAE78105E3D5B189890561
:106AC000E0D50E20DBE71220D9E7FF22F532064998
:106AD0000298085402986359091804481B1DF9F7D5
:106AE0004BFCFEBD1052FF1FDC76FF1F556D0211DF
:106AF000F8B50446002000900E461020F9F7F8FA89
:106B0000544AA500515900280862515978D01746B7
:106B10008C6810223146F9F79DFA785901780029DE
:106B200062D1026A6069177B2146C307FF071431EF
:106B3000DB0FFF0F0C32BB4204D1C30702D001238D
:106B4000184301E040084000086017788307BF073A
:106B5000DB0FFF0FBB4204D1830702D5022318438A
:106B600001E0022398430860177843077F07DB0F93
:106B7000FF0FBB4204D1430702D50423184301E0B1
:106B80000423984308601788C305FF05DB0FFF0F38
:106B9000BB4205D1C30503D5FF230133184302E0EF
:106BA000FF2301339843086017888305BF05DB0F77
:106BB000FF0FBB4205D1830503D501235B021843B8
:106BC00002E001235B0298430860128843055205E6
:106BD000D70F0122DB0F9202BB4203D1430501D53F
:106BE000104300E0904308607078002809D0607876
:106BF000002806D01748052140592030017125E0B2
:106C000026E03079400708D4A07C400705D411491C
:106C1000012049592031087118E00E484259107876
:106C2000002802D02078317801E0217830780428DB
:106C300001D8042901D9182007E08B00C918064B98
:106C4000C918085C20321071002000900098F8BD2F
:106C50001320FAE71052FF1F467C021170B50C4654
:106C60000A460646054B022100F00AF8054621783F
:106C70003046FFF799FB284670BD0000C77102112E
:106C8000FEB51646054606226846028001811C466E
:106C90000846FBF7D9FA019000280ED0014630468D
:106CA000A047040005D169462846FBF7B3FA040063
:106CB00004D00198F9F776FA00E01324284600F092
:106CC00023F82046FEBD000070B50D4681000D483A
:106CD000405800280FD08468002C0CD020782870F1
:106CE00060786870A17C281D00F054F8207E28721E
:106CF0006069E86070BD102200212846F9F7CEF9DE
:106D000070BD00001052FF1FF8B504462020FAF7AE
:106D100075FB0D4E0546A700F059002812D0002D36
:106D200010D0C078FF2804D02946F9F7B5FB002819
:106D300008D006482A460455F35901190448DB1CBB
:106D4000F9F71AFBF8BD00001052FF1F9C77FF1FD8
:106D50008B6D021110B50078FFF7DEFB10BD00004F
:106D600070B5064C85006059002805D0C078F9F749
:106D7000A9FA6159FF20C87070BD00001052FF1FB2
:106D800010B51721FFF710FB10BD10B50078FFF705
:106D9000F7FF10BD10B502688B07920892009B0F99
:106DA0001A434C0704230260002C01DA1A4300E066
:106DB0009A43F823C9089A43C9000A43026010BDE8
:106DC000FFB587B017461020F9F792F9019010200F
:106DD000F9F78EF90090019800287DD000980028DE
:106DE0007BD0024601990798FDF7A8FC04007ED1EC
:106DF0001020F9F77DF902901020F9F779F906468D
:106E0000029800286BD0002E7CD038460F30050940
:106E100002D038070CD000E00125002029011039EC
:106E200000280898C9B205D04018324601991AE0E6
:106E30000120F3E7401884463A07120F002003A907
:106E40008023904202D267463F5C04E0904201D129
:106E50000B5401E000270F54401CC0B21028F0D39F
:106E6000324603A8009900F0C5FD102200210298C7
:106E7000F9F714F900276D1E0FE038070899000E86
:106E8000091803AA029800F0B5FD03A9029A079811
:106E9000FFF786FA7F1C04463FB2AF4202DA002CAD
:106EA000EBD011E0002C0FD103AA3146029800F07C
:106EB000A1FD03A9029A0798FFF772FA0446082277
:106EC00002990A98F9F7C6F80298002801D0F9F754
:106ED00021F9002E08D004E01AE017E007E013E0E3
:106EE00010E03046F9F716F90198002802D0019811
:106EF000F9F710F90098002801D0F9F70BF92046AE
:106F00000BB0F0BD1324E2E71324E2E71324EEE70D
:106F10001324EFE770B58CB015460E4604463022B8
:106F200000216846F9F7BAF8102221466846F9F7B9
:106F30004BF907A8032231460130F9F745F96846B5
:106F4000FFF726FA04460BA9032228460131F9F778
:106F50003BF920460CB070BDFFB5244D07468600B6
:106F6000A8598DB000281AD0C088FEF78FFE040003
:106F700018D005A93846FFF7A7FEA85901780029BF
:106F800012D005A90291006A0190FBF707FE00905C
:106F90000020FBF7F5FD0646A779E51D12E012205B
:106FA00011B0F0BD1420FBE7006A029005A8019023
:106FB000FBF7F4FD07460020FBF7E2FD0546A0794C
:106FC000E61D009009A9019800F063F90BA9029849
:106FD00000F016F9109804900BAB09AA02970196DD
:106FE00003950F990E9800F003F8D9E71052FF1F90
:106FF000FFB595B004461F463022002104A81E9E0E
:10700000209DF9F74BF81022214604A8F9F7DCF887
:10701000102200216846F9F741F8072268461799BF
:10702000F9F7D2F801A8072239460330F9F7CCF86E
:10703000002D01D0012000E0002069468873002E59
:1070400001D0012000E00020C8731022002110A808
:10705000F9F724F8062211A81F99F9F7B5F812A834
:10706000062202302199F9F7AFF808A81022064647
:107070001699F9F7A9F86946304600F03AF804A8DD
:10708000FFF786F904460CA910220D463046F8F7A2
:10709000E1FF10A9304600F02CF804A8FFF778F9BA
:1070A0000443102229462298F9F78EF8204619B099
:1070B000F0BD70B50C468CB0164601461D46102238
:1070C0006846F9F781F80822214604A8F9F77CF808
:1070D0000822314606A8F9F777F86846FFF758F90D
:1070E00004461022284608A9F9F76EF820460CB08D
:1070F00070BD10B5002203780C78521C63400370F9
:10710000D2B2401C491C102AF5D310BD10B500297D
:107110000BD0002809D006220A704B1C0146102211
:107120001846F8F797FF002010BD022010BD10B5DB
:1071300000290DD000280BD009220A704B1C0178C1
:107140001970411C0622581CF8F784FF002010BD5E
:10715000022010BD10B500290BD0002809D008224C
:107160000A704B1C014610221846F8F773FF0020E6
:1071700010BD022010BD10B50346002910D0002B11
:107180000ED007200870481C197801701988082251
:10719000090A4170991C801CF8F75CFF002010BDA3
:1071A000022010BD10B500290BD0002809D0032201
:1071B0000A704B1C014610221846F8F74BFF0020BE
:1071C00010BD022010BD002907D0002805D00522DF
:1071D0000A7000784870002070470220704710B590
:1071E00000290BD0002809D004220A704B1C01464C
:1071F00010221846F8F72EFF002010BD022010BD07
:107200000A4610B50146012000F001F810BD70B526
:107210000C46002A3BD0002C39D0107020785070DA
:1072200060789070D51C201DFFF790F82870207AA8
:107230006870A089C005C00FA870A1898905C90F11
:1072400049000843A870A1894905C90F890008436E
:10725000A870A1890904C90EC9000843A870207B41
:10726000C007C00FE870217B8907C90F4900084398
:10727000E870217B4907C90F89000843E870217B2A
:107280000906C90EC9000843E870002070BD02203D
:1072900070BD0A4610B501460220FFF7B8FF10BDC9
:1072A00010B500290BD0002809D00A220A704B1C07
:1072B000014610221846F8F7CDFE002010BD02202E
:1072C00010BD10B50B46002808D0002B06D0411C7D
:1072D00010221846F8F7BEFE002010BD022010BD97
:1072E00010B50B4600280AD0002B08D04178197041
:1072F000811C0622581CF8F7ADFE002010BD0220AC
:1073000010BD10B50B46002808D0002B06D0411C3C
:1073100010221846F8F79EFE002010BD022010BD76
:1073200010B50B4600280DD0002B0BD08278417889
:10733000120289181980C11C0822981CF8F78AFECD
:10734000002010BD022010BD10B50B46002808D04B
:10735000002B06D0411C10221846F8F77BFE0020B7
:1073600010BD022010BD002809D0002907D04078A8
:107370000870092805D8002803D000207047022093
:1073800070471820704710B50B46002808D0002B16
:1073900006D0411C10221846F8F75CFE002010BDF4
:1073A000022010BD70B50C4600281DD0002C1BD04B
:1073B0004178217081786170C178051D201DFFF72B
:1073C000E9FC287820726978FF22E0680132904356
:1073D000CA07D20D104301228B075202AD1CE06098
:1073E000002B03DA104302E0022070BD9043214AD3
:1073F000E0604B0701D5104300E090431F22D2020A
:10740000C9089043C9020843E06029784008CA07C8
:107410004000D20F10438B070222E060002B01DAFC
:10742000104300E090434B070422E060002B01DA98
:10743000104300E09043F822C9089043C900084374
:10744000E0602120F9F7DAFF217A884205D822206E
:10745000F9F7D4FF217A884201D2122070BD20783A
:10746000042802D86078012801D9182070BD0020B6
:1074700070BD00000004000010B50A46002807D0C7
:10748000002A05D041781046FFF784FC002010BD8B
:10749000022010BD10B50B46002808D0002B06D0E6
:1074A000411C10221846F8F7D5FD002010BD02201F
:1074B00010BD000070B515460E460724FEF7E6FB2A
:1074C000002807D042790D49002A05D0012A09D0A9
:1074D000052070BD082070BD094A127812070BD52F
:1074E000896800E04968002906D00B68002B03D0AA
:1074F0002A46314698470446204670BD1052FF1F69
:107500003551FF1FF8B5124C0646850060590F46ED
:1075100041780C291AD1C06E002806D11C20F8F73A
:10752000E7FD61590028C86610D060591022C06E6E
:107530003946F8F78FFD3046FEF714FF6159C96EE2
:10754000887661590D2048700020F8BD0720F8BDED
:107550001052FF1F70B5104C05468600A0594278A6
:107560000F2A01D0072070BD006F06221030491C81
:10757000F8F770FDA0598168898A490506D5016A26
:107580008989490502D51021417003E00021284670
:10759000FEF70AFF002070BD1052FF1F70B50F4CA0
:1075A000850060590E4641780E2901D0072070BD34
:1075B000006F002806D11620F8F79AFD61590028BF
:1075C000086705D060591022006F3146F8F742FD78
:1075D00061590F204870002070BD00001052FF1F3D
:1075E000FEB5054640882A4B86009B590024002B97
:1075F00004D0DD88854214D00820FEBD01290ED1BB
:107600001446101DFEF7A2FEE1680291217A009057
:1076100001916378227869880020FCF73FF8002008
:10762000FEBD1B78012B09D00B00F8F74FFD0B2E88
:10763000092E0D122A161A1E22262E000720FEBD24
:10764000114600F0ABF802E0114600F055F8044690
:107650001CE0114600F076F8F9E71146FFF752FFFB
:10766000F5E7114600F016F8F1E71146FFF796FF2F
:10767000EDE71146FFF76EFFE9E7114600F0EAF883
:10768000E5E71178FEF790FE00E007242046FEBDF6
:107690001052FF1F70B5174C05468600A059C26EE8
:1076A000002A02D040780D2801D0072070BD08883C
:1076B0001082A0590822C06E891C1230F8F7CAFC4B
:1076C000A15988684069820505D50A6A92899205A0
:1076D00001D50E2006E0400506D5086A80894005E0
:1076E00002D51020487003E000212846FEF75CFE1A
:1076F000002070BD1052FF1FF8B5114C07468500E1
:107700006059002610224530F8F7A4FC61594878EA
:10771000042812D00B460A462533353238460C3140
:10772000FFF71AFC3846FEF787FE002800D008262F
:107730006159052048703046F8BD0320FAE7000083
:107740001052FF1FF0B5144C07468500605985B0F4
:10775000002610225530F8F77DFC61596B460A4629
:10776000553238460C31FFF7F7FB61591022684655
:107770004531F8F77BFC012803D00426304605B0DC
:10778000F0BD3846FEF7A2FE002801D00826F5E736
:10779000615906204870F1E71052FF1FF8B5044602
:1077A0000026FFF7A5F9002804D018284ED0082697
:1077B0003046F8BD2046FEF755FEA500244C605922
:1077C0008168897CC90709D0016A09798907890F0D
:1077D000012903D1017F012211430177605924213E
:1077E000095C042702291ED003291CD004291AD0C1
:1077F000012901D00529DBD10221417060592421E2
:10780000095C01291CD0816810220C30891CF8F712
:1078100021FC6059017F39430177605910213530CF
:10782000FEF740FEC4E7022900D00121C088FBF723
:107830007FFA6059017F3943017760594770B7E794
:10784000102200210C30F8F729FCE6E70326AFE709
:107850001052FF1FF8B5134C0646850060590F46BD
:1078600000281CD0406F002806D11420F8F740FCF7
:1078700061590028486710D060591022406F39467E
:10788000F8F7E8FB61590020496FC0430861002107
:107890003046FEF789FD0020F8BD0820F8BD07201E
:1078A000F8BD00001052FF1F30B5094B0CE00C78FA
:1078B0005D6824092C5D04700C785D682407240F32
:1078C0002C5D4470801C491C521EF0D230BD00005B
:1078D000DC4EFF1F70B504460079BEB0C0072CD047
:1078E00060881749FAF712F9C0070226154D0028DB
:1078F0000ED0134800221030418D6846018046802A
:10790000698801710912417160886946FAF772FA53
:107910000B4960880831FAF7F9F8C0070DD008481C
:1079200069465030408B08804E80A888087100124C
:10793000487160880022FAF75DFA3EB070BD000021
:10794000F44EFF1FDE58FF1F70B5049C0020002C72
:1079500001D00B2070BD49680D4E0C784978022586
:10796000090261188CB20B49B44204D11D808B7896
:107970001370498807E0064E761CB44206D11D807C
:107980000B79137089880912517070BD0A2070BD7F
:107990006E2A0000DE58FF1F7CB515464A68069C1B
:1079A000167852781202B218104E92B2F24209D1F1
:1079B00001220192DBB200942A46F9F74DFF040040
:1079C00003D000E00A2420467CBD697828780902AB
:1079D0004018074980B209680029F4D0002802D075
:1079E00001208847EFE70220FBE70000FED6FFFFFB
:1079F000F04EFF1F30B50023C45CCD5C6C40D45406
:107A00005B1CDBB2102BF7D330BD0000030000007D
:107A100000000000000000000001020307090A0B3B
:107A20000E0F101112141718191A1B1F20212200F3
:107A30000201000504000807000B0A001716001DCC
:107A40001C010201010504010E0D011110011413A6
:107A5000011716011A19020201020B0A020E0D0289
:107A60001110021413021716030504030807030B71
:107A70000A030E0D000D000E00100011001300147B
:107A800001070108010A010B011C011D0204020586
:107A9000020702080219021A021C021D0301030256
:107AA00003170000020000000C7C0211D5470211F0
:107AB000F148021100000000020000000E7C0211DB
:107AC0000000000085450211000000001A186E2A0F
:107AD0006F2A000002000000CC7A021149790211DD
:107AE000997902110000000000030103020303035F
:107AF0000402050206020700080309030A030B0338
:107B00000C000D000E030F031003110013031403E8
:107B100015031603F1590000FD2400004146010041
:107B20004D210211652302117D150211251E02113E
:107B3000C5110211B1180211951002110A0A182478
:107B40002A252A262A272A282A292A000200000074
:107B50003D7B021154484232003030303100563003
:107B60002E340054757961006769746875622E63FC
:107B70006F6D2F70767678003D29021100000000AD
:107B8000000000000F18192A02000000847B021177
:107B9000BD270211F527021100000000FB349B5F96
:107BA000800000800010000000000000910D021114
:107BB000F1390211030E02113D3A0211BB0D0211FF
:107BC000113A0211DD0E02116D3B02115D0F02111F
:107BD000E13B0211BB0E0211E13B0211190F021130
:107BE000993B0211DD0E0211253B0211750F0211A6
:107BF000953C02110000000000000000830E0211FD
:107C0000953C0211A90D02110D3A0211001801183C
:107C10000028012802280328002901290229032914
:107C200004290529002A012A022A032A042A052AEE
:107C300006290729082900000000000000000000B4
:107C4000000000000087010102010201010201029F
:107C50000303040103010101010103030201030005
:107C60003031323334353637383941424344454672
:107C7000000000005048592B36325858504C55538C
:087C8000303530340000000033
:020000041FFFDC
:1000000000000000715E0211147B02113C7B0211A2
:10001000784FFF1F000000000000000000000000FB
:1000200000000000000000000000000000000000D0
:1000300000000000000000000000000000000000C0
:1000400000000000000000000000000000000000B0
:1000500000000000000000000000000000000000A0
:100060000000000000000000000000000000000090
:100070000000000000000000000000000000000080
:100080000000000000000000000000000000000070
:100090000000000000000000000000000000000060
:1000A0000000000000000000000000000000000050
:1000B0000000000000000000000000000000000040
:1000C0000000000000000000000000000000000030
:1000D0000000000000000000000000000000000020
:1000E0000000000000000000000000000000000010
:1000F0000000000000000000000000000000000000
:1001000000000000000000000000000000000000EF
:1001100000000000000000000000000000000000DF
:1001200000000000000000000000000000000000CF
:1001300000000000000000000000000000000000BF
:1001400000000000000000000000000000000000AF
:10015000000000000000000000000000000000009F
:10016000000000000000000000000000000000008F
:10017000000000000000000000000000000000007F
:10018000000000000000000000000000000000006F
:100190000939FF1FAD39FF1F0547FF1F0000000091
:1001A000000000000000000000000000000000004F
:1001B000000000000000000000000000000000003F
:1001C000000000000000000000000000000000002F
:1001D000000000000000000000000000000000001F
:1001E000000000000000000000000000000000000F
:1001F00000000000000000000000000000000000FF
:1002000000000000000000000000000000000000EE
:1002100000000000000000000000000000000000DE
:1002200000000000000000000000000000000000CE
:1002300000000000000000000000000000000000BE
:1002400000000000000000000000000000000000AE
:10025000000000000000000000000000000000009E
:10026000000000000000000000000000000000008E
:10027000000000000000000000000000000000007E
:10028000000000000000000000000000000000006E
:10029000000000000000000000000000000000005E
:1002A000000000000000000000000000000000004E
:1002B000000000000000000000000000000000003E
:1002C000000000000000000000000000000000002E
:1002D000000000000000000000000000000000001E
:1002E000000000000000000000000000000000000E
:1002F00000000000000000000000000000000000FE
:1003000000000000000000000000000000000000ED
:1003100000000000000000000000000000000000DD
:1003200000000000000000000000000000000000CD
:1003300000000000000000000000000000000000BD
:1003400000000000000000000000000000000000AD
:10035000000000000000000000000000000000009D
:10036000000000000000000000000000000000008D
:10037000E53AFF1F00000000000000000000000040
:10038000000000000000000000000000000000006D
:10039000000000000000000000000000000000005D
:1003A000000000000000000000000000B70502117E
:1003B000000000000000000000000000000000003D
:1003C000000000000000000000000000000000002D
:1003D000000000000000000000000000000000001D
:1003E000000000000000000000000000000000000D
:1003F00000000000000000000000000000000000FD
:020000041FFFDC
:10183800B07BFF1F1119FF1F81840000F1280000F1
:101848000000000000000000000000000000000090
:101858000000000000000000000000001D19FF1F2C
:101868000000000000000000CD8400002119FF1FC7
:101878002319FF1F2519FF1F2719FF1F2919FF1FEC
:101888002B19FF1F2D19FF1F2F19FF1F3119FF1FBC
:101898003319FF1F3519FF1F00000000000000006A
:1018A8000000000000000000000000000000000030
:1018B8000000000000000000000000000000000020
:1018C8000000000000000000000000000000000010
:1018D8000000000000000000000000000000000000
:1018E80000000000000000000000000000000000F0
:1018F8000448854600F020F800480047F95D0211C9
:10190800C046C046B07BFF1F0948804709480047CA
:10191800FEE7FEE7FEE7FEE7FEE7FEE7FEE7FEE797
:10192800FEE7FEE7FEE7FEE7FEE7FEE7FEE700006C
:101938000D27FF1FF918FF1F064C0125064E05E06D
:10194800E36807CC2B430C3C98471034B442F7D3D8
:10195800FFF7D2FF804DFF1FB04DFF1F70B58C18E9
:101968000578401C6B075B0F01D10378401C2A11D6
:1019780006D10278401C03E006780E70401C491C12
:101988005B1EF9D12B0705D40023521E0DD40B7012
:10199800491CFAE70378401CCB1A921C03E01D7817
:1019A8000D70491C5B1C521EF9D5A142D8D30020EA
:1019B80070BD000003B40148019001BD75A9000085
:1019C80003B40148019001BDF9A6000003B4014821
:1019D800019001BDA1AF000003B40148019001BD11
:1019E8009DA9000003B40148019001BD75110000D4
:1019F80003B40148019001BDDD3F000003B4014874
:101A0800019001BD8944000003B40148019001BD63
:101A18002144000003B40148019001BD750F000086
:101A280003B40148019001BD1130000003B401481E
:101A3800019001BD53B9000003B40148019001BDF4
:101A4800C95C010003B40148019001BD19070100F8
:101A580003B40148019001BDBD0B010003B4014866
:101A6800019001BDDD0C010003B40148019001BDE6
:101A7800DD0A010003B40148019001BD01340100F1
:101A880003B40148019001BD0934010003B40148C1
:101A9800019001BD0534010003B40148019001BD66
:101AA800F535010003B40148019001BDF935010085
:101AB80003B40148019001BDE917010003B40148CE
:101AC800019001BD6137010003B40148019001BDD7
:101AD80001D7000003B40148019001BD6DF6000074
:101AE80003B40148019001BD7912010003B4014813
:101AF800019001BD4DF9000003B40148019001BDFA
:101B0800C1F7000003B40148019001BD61890000DC
:101B180003B40148019001BDA9D8000003B40148ED
:101B2800019001BDB352010003B40148019001BD09
:101B38000D52010003B40148019001BD8B52010010
:101B480003B40148019001BDC1A5000003B40148D8
:101B5800019001BD9D6A000003B40148019001BDD8
:101B6800116E000003B40148019001BD8D82000090
:101B780003B40148019001BD090E000003B40148F7
:101B8800019001BD0189000003B40148019001BD25
:101B9800E1AC000003B40148019001BDE53A010041
:101BA80003B40148019001BD496D010003B4014827
:101BB800019001BD3D71010003B40148019001BDD0
:101BC800156B010003B40148019001BD016C0100CF
:101BD80003B40148019001BDBD5C010003B4014894
:101BE800019001BDD1AE000003B40148019001BDD0
:101BF800CD4C010003B40148019001BD154D010011
:101C080003B40148019001BD350E000003B401483A
:101C1800019001BDA96F010003B40148019001BD05
:101C28009573010003B40148019001BDE94C01001E
:101C380003B40148019001BDB30E000003B401488C
:101C4800019001BD21A9000003B40148019001BD24
:101C5800ADAE000003B40148019001BDC54C0211AE
:101C680003B40148019001BDC56D010003B40148EA
:101C7800019001BD51B8000003B40148019001BDB5
:101C880085C1000003B40148019001BDE9D40000FA
:101C980003B40148019001BDF9ED000003B4014807
:101CA800019001BDE9F6000003B40148019001BDAF
:101CB80075F8000003B40148019001BD19FA00004D
:101CC80003B40148019001BDE90B010003B40148C8
:101CD800019001BD6D0B010003B40148019001BDE5
:101CE800C115010003B40148019001BDCD0C0100EC
:101CF80003B40148019001BD71B0000003B401486C
:101D0800019001BDD9B0000003B40148019001BDA4
:101D18005976010003B40148019001BDED6B010043
:101D280003B40148019001BD8937010003B401489B
:101D3800019001BD2D11010003B40148019001BDBE
:101D48008914010003B40148019001BDC9A900002C
:101D580003B40148019001BDD544010003B4014812
:101D6800019001BD2D6C010003B40148019001BD33
:101D78007997000003B40148019001BD8552010024
:101D880003B40148019001BDEDA5000003B401486A
:101D9800019001BD6911010003B40148019001BD22
:101DA8008512010003B40148019001BD8D110100A5
:101DB80003B40148019001BDE512010003B40148D4
:101DC800019001BDF90D0100F8B52F4C20780728C6
:101DD80059D82E48027801212D480904002AC26BDF
:101DE80016D08A43C263252001F074F929482023BC
:101DF8000168194301605806016804224D0714213F
:101E0800002D0FDB0568154305606D46297005E058
:101E18000A43E7E76E4635786D1E35706D462D78B6
:101E2800002DF7D1C5686D0709D4C5681543C5608D
:101E38006A4611706E463278551E3570FAD2C268FD
:101E48009A43C2606A46117003E06D462A78521EB2
:101E58002A706A461278002AF7D1C2681A43C2600B
:101E68006846017003E069460878401E08706846B5
:101E780000780028F7D10848017D217841601D21AC
:101E880001707621C160F8BDB04DFF1F744FFF1F70
:101E980000F00040BC4DFF1F002000400446FFF743
:101EA80089FD0A49C86940229043C8612046FFF766
:101EB80087FD01F09BFC05480021C03041600421EA
:101EC80001600120FFF782FDFEE7000000F00040FE
:101ED80010B5FFF76FFD0A480468094A41178032B8
:101EE800116008490160FFF777FD204610BD10B565
:101EF8000446FFF75FFD02480460FFF76DFD10BD63
:101F080000E100E01000100038B5044600F09EF92A
:101F18000146684601704470210A81706A460321AF
:101F28000248FFF75FFD002038BD00001B200000BD
:101F380038B5044600F0B0F90146684601704470AF
:101F4800210A81706A4603210248FFF74BFD0020F1
:101F580038BD00001A20000070B50124A407A3684A
:101F680010252B43A360FFF743FDA068A843A0609A
:101F780070BD0000FFB5064601208007816881B06A
:101F88001D46102211438160554F002038603046AD
:101F9800D730FFF733FD9D20800034468059FF3647
:101FA800CA3401360028306822462CD00121FFF7B8
:101FB8002BFD4B4F2078F863641C2046FFF72AFD61
:101FC80000BA000AE17800020843B863241D2046DD
:101FD800FFF720FD00BA000AE178000208437863A1
:101FE800241D2046FFF716FD00BA000AE17800021A
:101FF800084338630398029900020843F860039F76
:1020080000243F1D0EE00021D1E72819401CFFF7EE
:1020180001FD0102285D0143324820180160241D9A
:10202800A4B23F1F042FF0DA032F04D0022F08D0E8
:10203800012F0CD011E02819FFF7ECFC0102090A66
:1020480006E0291948780A780102114300E0295D61
:10205800244820180160241DA4B20021214F02E069
:10206800E0190160241DFF2CFADD1D481E4A42605C
:102078000F220261012202604269002AFCD04269F3
:10208800930701D4520708D40120800782681021E1
:102098008A438260002005B0F0BD01600020039AE9
:1020A80011E0C11909682954401C80B20B0A2B544D
:1020B800401C0B0C80B22B54401C80B2090E2954D2
:1020C800401C80B2121F002AEBDC3068401C3060D4
:1020D80001208007826810218A4382600120DAE7A4
:1020E8000000044000010440080F0000FFB5054649
:1020F80001208007816881B01E461022114381604B
:10210800504F002038602846D730FFF777FC9D20D5
:1021180080002C464059CA3480350028E86F224692
:102128002BD00021FFF770FC464F2078F863641C21
:102138002046FFF76FFC00BA000AE1780002084366
:10214800B863241D2046FFF765FC00BA000AE17851
:10215800000208437863241D2046FFF75BFC00BAA1
:10216800000AE178000208433863039802990002E4
:102178000843F8600024039F0EE00121D2E73019DC
:10218800401CFFF747FC0102305D01432E48201830
:102198000160241DA4B23F1F042FF0DA032F04D0DE
:1021A800022F08D0012F0FD014E03019FFF732FCAE
:1021B8000102090A09E03119487809780002084340
:1021C80021496118086003E0315D1F48201801604B
:1021D800241DA4B200211C4B02E0E0180160241D5C
:1021E800FF2CFADD0F221748120242600F2202610B
:1021F800012202604269002AFCD00160039A002093
:10220800121D11E0C11809683154401C80B20C0A33
:102218003454401C0C0C80B23454401C80B2090E5B
:102228003154401C80B2121F002AEBDCE86F401CBE
:10223800E86701208007826810218A43826005B020
:10224800F0BD0000000004400001044010B5114A30
:10225800A1218900126841438C189D2189000959E0
:10226800012901D00C2010BDFFF7DAFB0028FAD1B4
:10227800E01DF93002790621012A06D041710D21AD
:102288002046FFF7D3FB002010BDFF202130015569
:102298000221F5E73409FF1F70B50D46134AA12145
:1022A8008900126841438C189D2189000959012928
:1022B80001D00C2070BD002D16D0FFF7B1FB00280F
:1022C800F8D110210B1A2A5C1B19E033401CC0B24C
:1022D8009A711028F6D30121F820015505212046CE
:1022E800FFF7A4FB002070BD122070BD3409FF1F4A
:1022F800F8B5FFF7A1FB564908600420FFF7A2FBD9
:10230800FFF7A6FB0646C00715D052490020086013
:1023180051480078012811D0032813D0042815D07B
:10232800022817D0052819D0FFF798FB4B4F044611
:1023380001281AD01EE0FFF797FBF8BD3046FFF7DB
:1023480099FB0EE03046FFF79BFB0AE03046FFF7AB
:102358009DFB06E03046FFF79FFB02E03046FFF7A3
:10236800A1FB40B20128E8D04FE0387805280BD00F
:10237800062809D03A483B4D0078022808D005289D
:1023880006D0022C0ED005E0304601F0F3FE3CE00A
:10239800022C02D0012C11D014E0A87B002805D013
:1023A800022803D03878052804D00BE0304601F025
:1023B800F9FE15E0304601F0E9FE11E0012807D0EA
:1023C800062809D03046FFF773FB022C08D01CE022
:1023D800304601F0FFFE18E0304601F0EFFE14E051
:1023E8003878012811D170050FD4687BC10701D056
:1023F800252004E0800701D5262000E02720297D3C
:10240800814202D93220FFF759FB154C2078042865
:1024180004D003280ED0072811D014E0FFF754FB8E
:10242800002810D0FFF756FB5820FFF759FB022071
:10243800207008E00C48807CFFF758FB03E00B484D
:10244800807BFFF759FB0320FFF7FCFAF8BD00007B
:102458009C09FF1F9809FF1F9009FF1F1C09FF1FF8
:102468002309FF1FA60BFF1FBC0BFF1FD40BFF1F69
:10247800F8B56F4D0028AB7916D0012B01D0032B8E
:1024880012D16C490A78FF2A0ED14A78FF2A0BD15B
:102498008A78FF2A08D1CA78FF2A05D10A79FF2A43
:1024A80002D14979FF2937D063490A78012A1DD01A
:1024B8000026624C0E702278092A77D00A2A75D035
:1024C8000B2A73D00C2A71D00D2A6FD0052A6DD033
:1024D800062A6BD0A97B00290AD0012908D0032934
:1024E80006D0022904D0042916D101E00C20F8BD39
:1024F800002B05D0012B03D0022B01D0032B0BD1CD
:10250800032901D0022902D16B88202B04D34C4F18
:1025180000286AD0012801D01220F8BDA888012817
:1025280044D0002A17D10B00FFF7ECFA0504081075
:102538000C082400012020701F200AE002202070CF
:10254800202006E004202070222002E003202070D2
:102558002120FFF777FA2078282101280DD00228BA
:102568000BD0042809D0032807D007280ED0082844
:102578000CD01BE026701E20EBE732480660297558
:10258800FFF7C6FA00281FD0AE800FE02E4840683B
:10259800808D80060AD52D480278002A06D1AA7BAC
:1025A800032A05D0022A03D0002A01D02120F8BD31
:1025B800022202702975140321463878FFF7AEFA13
:1025C80021463878FFF7B0FA0120A8802048007823
:1025D80000282AD01F48012102887D20C0004243DC
:1025E800C9033878FFF7A6FA1FE0FFF7E3F9AE80D2
:1025F8002078072808D0082806D026701648FFF744
:102608009FFA1E20FFF71EFA10480178002905D00E
:102618000670012149033878FFF780FAFFF7DCF9E3
:102628000121C9033878FFF779FA0020F8BD0000C6
:10263800A60BFF1F6B09FF1F1A09FF1F1C09FF1FAD
:102648001B09FF1F4809FF1F0851FF1F2309FF1F10
:102658002109FF1F2C09FF1F00100040F0B585B0AD
:1026680014468C4686460AAD87CD0D4E35780397BD
:102678006F4607C7224661467046FFF767FA35700E
:10268800012C01D0042C08D1064980240978CA01FC
:1026980005498B88A3431A438A8005B0F0BD000022
:1026A8001C09FF1F7809FF1F6C11FF1F10B5FB29BC
:1026B80008D8084B9A4205D81B2903D3FF2349336E
:1026C8009A4201D2302010BD034B19825A82FFF77B
:1026D80043FA10BD480800008410FF1F10B5FFF72B
:1026E80041FA02490020488010BD00000851FF1F30
:1026F800C106C90E012088400149086070470000E2
:1027080000E100E0024901480860704740787D0117
:102718000451FF1F10B57D21C003C900FFF728FA37
:10272800FFF72CFA10BD00008307FF22DB0E9A404A
:102738008907090E9940002808DB830809489B008F
:102748001B18186890430843186070470007000F6B
:102758000838830804489B001B18D869904308432D
:10276800D861704700E400E000ED00E0EFF303807B
:10277800704702E008C8121F08C1002AFAD1704742
:102788007047002001E001C1121F002AFBD17047E9
:102798000248C069002800D0004770474003FF1F67
:1027A8001CB569460120FFF7EFF9012000900348A6
:1027B800019000F075FA01201CBD0000BB0B000061
:1027C80004460DA0FFF7E6F911A0A16BFFF7E2F9A7
:1027D80013A0E16BFFF7DEF915A0216CFFF7DAF91A
:1027E8001748416817A0FFF7D5F91A48006800286C
:1027F80000D08047FEE700005B4861726420666194
:10280800756C742068616E646C65725D0A00000006
:102818004C522020203D203078253038780A00009E
:1028280050432020203D203078253038780A000099
:1028380050535220203D203078253038780A000047
:1028480000ED00E049435352203D203078253038D0
:10285800780A0000D84EFF1F10B500F0FFF9FFF707
:102868009FFF002802D00248804710BDFEE7000005
:10287800E1A20000F0B585B005460291002927D0F5
:10288800154F0024144E803F00230094022219465D
:1028980005200194FFF784F930698007FCD42020D3
:1028A8000090411E009101D30846FAE738680028D5
:1028B800FCDA012103A8FFF779F96846007B284074
:1028C80007D00520FFF75AF90298401E0290DBD185
:1028D800112005B0F0BD000080C80040F8B54E4892
:1028E8004068C043000603D53C20FFF747F9F8BD10
:1028F800FFF762F9484D0090803D2868012189045E
:1029080008432860E869454908402830E861032001
:10291800FFF734F9686AC703FF0B0320FFF72EF9A6
:10292800686AC403E40B0320FFF728F9686AC60342
:10293800F60BA74201D3204600E03846B04200D348
:102948003046A74201D3394600E02146B14200D2C1
:102958003146334ABA18C32A26D2314BDB439C424C
:1029680022D9304A94421FD29E421DD996421BD288
:10297800081A132818D2284842680C218A43426052
:102988004168FF221202914341601420FFF7F6F8D4
:1029980021488038416AC269C903C90B08239A4390
:1029A800C2612148C160F8BD274634460320FFF7BD
:1029B800E5F819488038406AC603F60BFFF7FCF8BB
:1029C8000099884201D3401A01E0401A401E174975
:1029D8008842AED31048416809040D0E4168FF22B1
:1029E800120291436A1C1206120C1143416041689D
:1029F8000C229143091D41600020FFF7E3F8642D84
:102A080002D3054800214160062D00D3062507485A
:102A1800A840FFF743FA8CE7C0F0004000FEFEFF35
:102A280091FCFFFF320400000851FF1FE40C000076
:102A3800F8B53D4840683C4C0006803C80210028A1
:102A480006DB6068084360600320FFF797F8F8BD6D
:102A5800364D0020686120680122920410432060EE
:102A6800334F60688021084360600320FFF786F8D1
:102A78006869401C68616068012109040843606056
:102A88000026E0692B4938404018E0610320FFF731
:102A980075F8606AE169C003C00B08229143E161DF
:102AA800E96806225143814201D3091A00E0411A1C
:102AB8003C2909D2E269012109048A43E26162687A
:102AC8008A4362602861F8BD761CF6B2052ED8D319
:102AD800E169012000048143E1616168814361602B
:102AE80068692E46052807D3BFF34F8F134912484C
:102AF800C860BFF34F8FFEE760688021884360603D
:102B08000320FFF73BF8E06938402830E0610320F4
:102B1800FFF734F8606AC003C00BF060E169082071
:102B28008143E1619DE70000C0F000400851FF1FAC
:102B380000FEFEFF280001000400FA0500ED00E099
:102B480001680A0508D11031044A0160527812035D
:102B5800914201D3891A016070470000E84DFF1FB8
:102B6800F0B58646080CFF268446002388B237460F
:102B78001C46194601228A4005461540CD402C19AD
:102B8800A4B2FF2F02D1012C00D18FB265462A4092
:102B9800CA40D21893B2FF2E02D1012B00D18EB2B7
:102BA800491C1029E6DB012C02D0102C08D009E0C2
:102BB800012B07D13001C019714608700220F0BD01
:102BC800102B01D00320F0BD0120F0BDF8B504465C
:102BD8000120FEF7D3FFFEF7FBFF1849184A0860EB
:102BE800966A184B1E60184BDF6A184D2D68AF4265
:102BF80002D2DB6AEB1A00E00023154D2B60331973
:102C0800D362536A2924E40323435362114A127896
:102C1800002A0FD0104A1378022B07D01378012B03
:102C280006D01278032A06D0C01E02E00F3800E052
:102C380008380860F8BD401FFBE70000E408FF1FE4
:102C480000F00040340AFF1F00100040180AFF1F60
:102C58001C0AFF1F1C09FF1F4A0AFF1F0349002007
:102C680048610349086048607047000040F0004030
:102C780040F1004010B5044607484068808DC00701
:102C880005D00648406AC003C00B01F00DFB204682
:102C9800FEF7A4FF10BD00000851FF1F40F00040E0
:102CA80070B58AB000241E4D049405942878012834
:102CB80006D004A90120FEF767FF002802D00020F3
:102CC8000AB070BD04980090059801901548816875
:102CD8000291C0681349039006AA10316846FEF7AE
:102CE80087FE104E10222036314606A8FEF77CFFDC
:102CF800002811D0012028700B4A31466846FEF79B
:102D080077FE04940020694605948200401C8C508C
:102D18000428FADB0120D3E7FF202870CFE7000062
:102D28000452FF1F00290011EC76FF1FF0B5504E2A
:102D3800504C9DB07168216071782171FF21A1719B
:102D48001021002561712F460922FF21E01DFEF7A1
:102D580051FF4E22002106A8FEF74CFF32E029035E
:102D680020681A914018102202A900F03FF9029930
:102D78002068814218D16946097B2279914213D192
:102D88006946497B627991420ED168467178807BA9
:102D9800491E884224DAA84201D1022700E003270D
:102DA80006A94855A0710BE01A99401800F0EAF9F5
:102DB8001022FF2102A8FEF71DFFFF2006A9485593
:102DC8006D1CEDB22179A942C9D8042F08D0A07989
:102DD8000125FF2807D0012F05D0002006AA24E0EE
:102DE80020201DB0F0BD00270DE0A7712068390331
:102DF800401810221F4900F00FF9002801D01F20A9
:102E0800EFE77F1CFFB22079401EB842EDDC0020BE
:102E180020742079401E607410206082357025E08F
:102E2800135C002B03D0401CC0B28142F8D8814209
:102E38001CD9401E0818FEF7E3FE617400203570A7
:102E480002466946009000F017F8002802D02128B1
:102E580002D004E0009901E0012109036182C0B2B7
:102E6800212803D0002801D02A20BAE70020B8E79B
:102E7800E84DFF1F1054FF1FF7B501248AB000204A
:102E88000E46274605909CE056480179407CC019BB
:102E9800FEF76EFEC8B2FF2C03D3FF3CA4B2FF2C92
:102EA80033D20A9A002A01D14E4A117400030290C3
:102EB80005980125002803D000200590601C06E035
:102EC800012C05D92819811EFF2917DA401E85B261
:102ED80002982901081807904248042201680798B7
:102EE800081804A900F082F80A9800280ED00128D2
:102EF80029D002283CD006200DB0F0BDFF200230BA
:102F0800401B201A84B20120059058E004988103E0
:102F1800890F04D0022902D003294CD10EE0010305
:102F2800890F012901D0012445E0000D0C21FEF78D
:102F38001FFE002900D0012144183CE00798000535
:102F4800000D306047E0049881038A0F04D0022AFC
:102F580005D0032A2FD142E0890F0229DFD1328818
:102F680081B292B29142DAD10C990798086032E0A6
:102F780004988103890F04D00229D0D003291AD1DB
:102F880029E00103890F012903D0306801240C309E
:102F98000BE0000D0C21FEF7EBFD002900D001210C
:102FA80044180C2031686043081830600C980C995C
:102FB8000068401C08606D1CADB2FF2D80D97F1CD5
:102FC800FFB209484078874200D25DE70A98002896
:102FD80003D0012803D000208EE721208CE725208C
:102FE8008AE700001054FF1FE84DFF1F10B5094C79
:102FF800636898420BD364782403E318834206D9A4
:10300800002904D0002A02D000F018F910BD2220AF
:1030180010BD0000E84DFF1F70B515460E4604466A
:10302800FFF7A4FB800601D0292070BD0949486834
:10303800844206D3497809030818A04201D9A00799
:1030480001D0222070BD2A463146204600F052F9B0
:1030580070BD0000E84DFF1F38B5FEF7ABFC01223C
:103068009207936A08240094002B01D101209062F2
:103078000A480221016000994D1E0095FBD20321E8
:1030880001600094641E0094FCD200210160002BB2
:1030980000D19162FEF7A0FC38BD000000C00040DE
:1030A800012189070122202804D28B68824093439A
:1030B8008B607047402805D24B6920388240934383
:1030C8004B6170476028FCD20B6A403882409343BA
:1030D8000B627047012292070121202804D29368CD
:1030E80081400B4393607047402805D253692038CC
:1030F80081400B43536170476028FCD2136A403803
:1031080081400B4313627047012110B589070122E2
:10311800202813D20346153B012B07D80A68202024
:1031280082430A600A6802430A6010BD0B68824045
:1031380093430B6008681043086010BD402814D200
:103148000346353B032B07D8CA6810208243CA6060
:10315800CA680243CA6010BDCB68203882409343D6
:10316800CB60C8681043C86010BD6028FCD24B6AA9
:103178004224201A824093434B62486A10434862B3
:1031880010BD0000F1B584B0FEF7A2FE0124A4072B
:103198000190A76AFEF70EFC2549022008606062CC
:1031A8000120A062FEF718FC224E30698007FCD48B
:1031B8002020204D0090803D0098411E0091FBD2B8
:1031C80028680028FCDA1C490120FFF753FB002877
:1031D80017D10498FEF71AFDC0B202903069800733
:1031E800FCD420200090411E009101D30846FAE744
:1031F80028680028FCDA10490320FFF73BFB002869
:1032080002D0112005B0F0BDFEF7D4FB084900201C
:10321800086003216162A062FEF7DEFB002F01D186
:10322800FFF71AFF0198FEF762FE0298EAE700002E
:1032380000C0004080C80040FFFFFF07F7B582B01C
:103248000646FEF745FE019070031121400B090662
:1032580040188D010090AF6A234800248168E81265
:1032680081420AD91F203446C004044005D01F48B3
:1032780044620168AA1311430160002F09D1FEF7C7
:1032880099FB1B490220086068620120A862FEF7CA
:10329800A3FB002004E000990A5C03990A54401C2F
:1032A80004998842F7D30026002F08D1FEF782FB45
:1032B8000F48066003206862AE62FEF78DFB0A487D
:1032C80081680120C004814208D9002C06D0074833
:1032D80046620268012109048A4302600198FEF7E8
:1032E80006FE002005B0F0BDDC4DFF1F00C8004001
:1032F80000C00040F7B584B0FEF7EAFD0190FEF784
:1033080059FB244F02203860440760620120A06204
:10331800FEF762FB204E30698007FCD420201E4D4A
:103328000090803D0098411E0091FBD2286800283B
:10333800FCDA1A490120FFF79DFA002818D104ABDE
:1033480007CBFEF769FCC0B2029030698007FCD455
:1033580020200090411E009101D30846FAE7286812
:103368000028FCDA0D490120FFF784FA002802D072
:10337800112007B0F0BDFEF71DFB002038600321C7
:103388006162A062FEF728FB0198FEF7B0FD029883
:10339800EFE7000000C0004080C80040FFFFFF07C3
:1033A80070B50F4900200978002916D00D4A01256B
:1033B800548A2D03AC420FD2507C1179127C4018EC
:1033C800801A401EFEF71CFCFF2000014143281B09
:1033D80040180C214843000970BD002070BD000052
:1033E800E84DFF1F1054FF1F10B5084A1378002B33
:1033F80001D0272010BD030501D1022901D20620E2
:1034080010BD51705060FFF791FC10BDE84DFF1FD3
:10341800FEB5002405460094FFF7A8F9800601D000
:103428002920FEBD21480078002807D06946284693
:1034380000F040F8002803D02520FEBD2720FEBD5F
:103448001B4D009928680422401801A9FFF7CEFDFA
:1034580001980C21000DFEF78BFB002900D00121FB
:10346800461803273F041CE02868009904224018E6
:1034780001A9FFF7BBFD01980099B843019028689E
:103488000422401801A9FFF7C7FD002801D01F201A
:10349800FEBD0098103000906846FFF751FB641C91
:1034A800A4B2B442E0D30020FEBD0000E84DFF1FE7
:1034B8001054FF1F08B500220092064A1278002A0D
:1034C80006D00A46009069460120FFF7D5FC08BDE2
:1034D800272008BDE84DFF1FFFB583B01C461646E0
:1034E8000F460025FFF742F9800602D0292007B0D1
:1034F800F0BD2248007800280BD0002F0BD0002EFA
:1035080009D069460398FFF7D5FF002805D0252084
:10351800EDE72720EBE72220E9E719480099006842
:103528000422401801A9FFF761FD002C02D0019880
:10353800000D20800198040DB44219D91CE00C2C10
:1035480001D30C2000E02046C6B20D487919026864
:103558000098001D10183246FFF748FDA01B84B2E2
:10356800009810300090A81985B26846FFF7E8FA6D
:10357800002CE4D10020BAE72620B8E7E84DFF1F69
:103588001054FF1FF7B588B014460546FFF7EEF84C
:10359800800602D029200BB0F0BD484800780028EA
:1035A80009D00998002804D0002C02D0444884424D
:1035B80003D92220EFE72720EDE7FFF7F1FEA0422D
:1035C80001D22320E7E705A92846FFF773FF002863
:1035D80006D12846FFF71CFF002801D00120DAE7B2
:1035E800009821050003000B0843009006946846E4
:1035F80005800321009809048843012149044018E3
:1036080000900C2C03D803218904084300902D4E08
:1036180000250C2C11D906980099A0422A4803D1FC
:1036280081430120800402E081430120C00408187E
:103638000C270C3CA4B200900BE000980103890F02
:10364800022901D0012902D11F4988430090E7B21D
:103658000024708A316804220818317C0903401854
:103668000590694601A8FEF7DDFA09983A4641191E
:1036780002A8FEF7D7FA3A1D01A90598FFF7CCFC76
:10368800002801D01F2086E7E81985B2708A012139
:10369800103080B20903708288420AD1307C3179B7
:1036A800401CFEF765FA707C814202D010207082BF
:1036B8003174002CADD100206DE70000E84DFF1FEC
:1036C800FF0F00001054FF1F00000C00F0B52F4C36
:1036D80085B02078012818D0FEF7FAFB2C4E03900D
:1036E80030698007FCD42027294D0097803D009839
:1036F800411E0091FBD228680028FCDA25490120E8
:10370800FFF7B8F8002821D102E0002005B0F0BD8D
:103718000020009003460146019003229F20FEF7F7
:103728003FFA032102A8FEF741FA30698007FCD46A
:1037380000970098411E0091FBD228680028FCDA07
:1037480014490120FFF796F8002801D01120DDE781
:103758000398FEF7CCFB6946887A497A0204090285
:103768000A436946097A0C4B0A43014662601139DB
:103778000122052904D811468140A160996103E01E
:103788000120C004A06098612270BEE7DC4DFF1FD5
:1037980080C80040FFFFFF078008FF1F08B504220C
:1037A80069460748FFF74AFD0098401C05D10548BF
:1037B80041690122920611434161002008BD0000C1
:1037C8001C18001100F00040074943090A78D20884
:1037D800D200002B02D00A70062070474007400F25
:1037E80002430A7000207047B54DFF1F0348C169A6
:1037F8001F2252049143C1610020704700F000402D
:103808000648C1691F2252049143054A127852079B
:10381800120B1143C16100207047000000F0004006
:10382800B54DFF1F10B578210848FEF701FA084882
:103838000078012803D0022804D0042804D1FEF718
:10384800FDF901E0FEF700FA002010BD8C53FF1FC0
:10385800B44DFF1F70B505461248122400780128A0
:1038680015D0042813D0FEF7A5F80F4800210C2224
:103878004A43825C002A11D0AA420CD10C23594336
:10388800012208184270FEF7D9F9002406E0FEF775
:10389800D5F9002070BD491C0A29E8DBFEF79CF821
:1038A800204670BDB44DFF1F8C53FF1F70B5124CDE
:1038B80000230C255D43655D854201D1072070BD5D
:1038C800002D04D05B1C0A2BF3DB032070BD0C25F4
:1038D8006B431B19094C25786E07ED086D1C760F94
:1038E800ED002E432670002BEFD000245C7018707A
:1038F8009A602046596070BD8C53FF1FB54DFF1F5D
:1039080070B5FFF77DFF0B480078C408641E0DD41E
:10391800094D20460C214843295C002908D040194C
:103928004068002800D08047641EF2D5002070BD92
:10393800122070BDB54DFF1F8C53FF1F70B5054693
:10394800164800240078012811D004280FD0FEF76B
:1039580031F80021124A0B4608460C267043165CC3
:10396800002E0FD0AE4205D18018437007E0FEF755
:1039780065F90DE080184078002800D0641C491CC7
:103988000A29E9DB002C05D0FEF758F9FEF724F8E0
:10399800002070BDFEF758F9F8E70000B44DFF1F8E
:1039A8008C53FF1F70B51B480121890742688A6044
:1039B800826801231A434A6117490A6BC260496B3E
:1039C800016100210420FEF7AFFE01211420FEF75B
:1039D800ABFE01211520FEF7A7FE01211720FEF7F7
:1039E800A3FE0C4E00240D4D761C0BE020460C2146
:1039F8004843295C00290BD040198068002800D072
:103A08008047641C3078C008A042EFDC002070BDFD
:103A1800122070BDB44DFF1F80F000408C53FF1F73
:103A280005490448086005490860054900204860C0
:103A380070470000841E0000140AFF1F380AFF1F89
:103A4800C0F0004010B5FEF707FF10BD70B5174C69
:103A58004025012819D0002816D100210A20FEF798
:103A6800F9F800210B20FEF7F5F8E06903210902B7
:103A78000843E061E069A843E06160690B21400107
:103A8800400909074018606170BD6069052140015F
:103A98004009C90640186061E069054908400549C0
:103AA8004018E061E0692843E06170BD00F0004023
:103AB8007F00FEFF80FD010010B5064A10705160BE
:103AC80000F012F8044A00211320FFF7EFFE00204F
:103AD80010BD0000D44DFF1FF13AFF1F08B50020AC
:103AE80000906846FEF76CFEF8B51F481F4942680B
:103AF8008A4201D1012100E00021009100780023D1
:103B08000121FEF7ADF81B491948886319480025BB
:103B180040300561102141610226866188031649FB
:103B28000860BFF34F8FBFF36F8F14480168FF22FF
:103B380012049143B20511430160642000904120B2
:103B4800FFF7C8FA4020FFF7C5FA740766620098C5
:103B5800411E0091FBD203206062FFF77DFAA56247
:103B6800FFF7B4FDF8BD0000D44DFF1F6B0001083E
:103B7800050001FF00C8004080E100E010E400E01B
:103B880070B50D4E7068FF300130056AFDF712FF01
:103B980000F0B6FB71680024FF310131496A491908
:103BA800814204D205490968002900D1441BFDF768
:103BB80013FF204670BD00000851FF1F9809FF1F22
:103BC80070B50D460446282910D1A420005BE18871
:103BD800401A0B4980B2884208D321466A3105222F
:103BE8000E46481FFEF700F8002804D02946204654
:103BF800FEF73CF870BD31462046FEF73DF870BD33
:103C0800FF7F000010B5002901D0FEF73BF810BD7A
:103C180070B50024FDF7CEFE0D484068FF3019301E
:103C280060C800F06DFBA919814203D209480068F9
:103C380000280AD008490420087008488169491CEE
:103C48008161FDF7C9FE204670BD0124F9E7000037
:103C58000851FF1F9809FF1F2309FF1FFC0FFF1FB3
:103C680010B5FEF715F80649A1228978920051434C
:103C7800044A12688918044A498C518010BD000012
:103C8800300DFF1F3409FF1F0851FF1F70B51F4873
:103C9800012201781E4D002915D01E48A1218078E7
:103CA800890048431C491D4C096822704618207831
:103CB80000F0D0FCA87B00281AD003281BD00228CB
:103CC8001CD0002070BDA97B002904D0032904D092
:103CD800022904D005E0027003E0042100E003217A
:103CE8000170FDF715FF0E4900200870012070BD16
:103CF800FDF7D4FF04E0FDF7D7FF01E0FDF7DAFF99
:103D0800FF36FF360236317B217070BD1C09FF1F5C
:103D1800A60BFF1F300DFF1F3409FF1F490AFF1FA5
:103D28002309FF1F70B5264D264E2868002804D0A9
:103D3800FDF7C6FF2978C84004E0FDF7C1FF3168E8
:103D4800FDF716FF04462868002804D0FDF7BEFFDB
:103D58002978C84004E0FDF7B9FF3168FDF708FF8E
:103D68001949A122897892005143184A184B1268C0
:103D780089180D78174A002D17D0FF31FF3102310D
:103D88004C6C1548641C4C6400689968884201D3DF
:103D9800401A02E0114B591A0818D2381060012C49
:103DA80002D1FF30F530106070BDFF31FF310025C2
:103DB80002314D645968201AC9684018F3E70000B9
:103DC8001C08FF1F1808FF1F300DFF1F3409FF1FB5
:103DD8000851FF1FA009FF1F9C09FF1FFFFF3F009D
:103DE800F3B506466548A1218078890048436449AF
:103DF80083B00968A12244182046FF3021305F496A
:103E080000908978920051435D4A407D12680025F0
:103E18008F18FF37813732281DD022281BD0F86A27
:103E28000168002909D08188001D090A891CFDF74D
:103E380053FFF96A002001250860FDF753FF049934
:103E48002746FF370880C137387C002821D0B04288
:103E58001FDC002014E04B49012008600020F96AAB
:103E680001250860E9E780000019FF308130006B08
:103E78008188001D090A891CFDF72EFF0198401C46
:103E88000190397C8142EEDCC8B2361A451900200F
:103E980038743D490020C870FF20AD3000590168D2
:103EA800002903D00079C04380071ED00098C07D48
:103EB80000281AD00098807D002816D1387CB0429E
:103EC80013DAFF204930005B010A2046FF304930F1
:103ED800891CFDF701FF00990020C8750098012191
:103EE800817529486D1CC170761E387C002802D067
:103EF800284605B0F0BD2046FDF7FAFE00900028E0
:103F080021DD002E1FDD002718E02046FDF7F6FE14
:103F180080000019FF300130C06E8188001D090A39
:103F2800891CFDF7D9FE2046FDF7EEFEE01DFF30A7
:103F3800FA30016A6D1C491C7F1C01620098874297
:103F480001DAB742E1DB092080012018817E0029CF
:103F580011D0017D00290ED0428E002A0BD0817F1E
:103F6800914202D2491C817705E0002181771A210C
:103F78002046FDF75BFDA8B2BBE70000300DFF1F30
:103F88003409FF1F00140340E010FF1F70B54E48AE
:103F98000068012803D14D48816D491C8165FDF7F2
:103FA8004BFD4B4D4B49A8604B4841610124C4600F
:103FB80004602878002806D0062248494848FDF7BA
:103FC80031FE002028704749486B474AC0B2127832
:103FD800002A17D1454A0023D356002B444BD35609
:103FE80006DB1B04002555572A029A18121808E008
:103FF800FF331B04002555572A029A183D4B121807
:10400800D2184A63022801D2022002E0502800D9BF
:104018005020394A1278022A11D0384A1578384B7C
:104028001E78B5420FD915781B78EB1A801E401000
:10403800434310784001C01A1030401104E0314A5F
:104048001578314BECE710784A69120A12021043CE
:104058004861FDF703FD0546052801D0042D1ED152
:104068002A480078002806D029480078002802D07D
:104078000020FDF74FFE2748A1218078890048439A
:10408800254909684018FF30FF300230007B0428BA
:1040980001D0032803D1FF205F30FDF721FD022D59
:1040A8000ED11E480078012807D0032805D0022821
:1040B80003D01B480078022802D16C20FDF710FDC0
:1040C8001848C48270BD00009809FF1FFC0FFF1F2D
:1040D8000851FF1FFF3F000000100340D50BFF1FD2
:1040E8007211FF1F800003408C09FF1F680AFF1F21
:1040F80000000000FFFE0000490AFF1F440AFF1FDE
:10410800450AFF1F460AFF1F470AFF1FF908FF1F3E
:104118002209FF1F300DFF1F3409FF1F1C09FF1F55
:104128002309FF1FBC0BFF1F0A48094901600B49FF
:10413800094A4A630A4A0A630A4A82600A4A8A633F
:10414800064A0A49803251610949C1627047000034
:104158006526FF1F4000FF1F893BFF1FC001FF1F8F
:10416800193CFF1F7924FF1F953CFF1FF541FF1FD6
:10417800693CFF1F10B504490968002901D0884728
:1041880010BDFDF795FC10BD8002FF1F10B5044956
:104198008968002901D0884710BDFDF789FC10BD4A
:1041A8008002FF1F10B504494968002901D08847DB
:1041B80010BDFDF77DFC10BD8002FF1F10B504493E
:1041C8000969002901D0884710BDFDF771FC10BDB1
:1041D8008002FF1F10B50449C968002901D088472B
:1041E80010BDFDF765FC10BD8002FF1F10B50D491D
:1041F800A1228978920051430B4A12688918242217
:10420800535C0A4A5288934209D2D21A084BC969A8
:104218005A435143421C02D0C82800D04018FDF729
:104228007FFD10BD300DFF1F3409FF1F0851FF1F10
:1042380071020000F8B51B484168802211434160B3
:10424800184D0A260027803DE86940084000E861CB
:104258000620FDF793FC134CC03CA069802108435D
:10426800A061E86901210843E86102E00820FDF740
:1042780085FCA86A800504D43046761EF6B200286C
:10428800F4D1002E07D0286A7E21C70BA0690F4001
:1042980088433843A061A16980208143A161380621
:1042A800400EF8BDC0F00040124B10B512497E22F6
:1042B80098420AD98B695B069B0E06D088698B6980
:1042C8004006800E9343401E0CE00C4B98420FD2E0
:1042D800886910407E280BD288698B694006800E59
:1042E8009343401C400003438B610320FDF746FCC9
:1042F80010BD00000B20000000F00040FD1C000075
:1043080010B5FDF799FB07484068062807D306490A
:10431800096801221205114201D1800810BD002050
:1043280010BD00000010004000E200E0F8B50024D5
:104338000C4E05460527A000801901686846FEF75F
:104348000FFC022805D0002C02DD012800D1032033
:10435800F8BD3A1B69460978641CA954062CEADBA7
:10436800F8BD00000009001110B5084906480860AA
:104378000749086000F0AAFA064A0121582000F00F
:1043880015FAFFF757FF10BD841E0000140AFF1F1F
:10439800380AFF1F600AFF1F30B53848016801223C
:1043A8009204114301604168032212069143344A82
:1043B80013781B06194341604368032189058B4321
:1043C80030490C78A40523434360436860242343A1
:1043D80043601378022B08D01378012B05D00B7893
:1043E800022B02D00B78012B04D14368FF2401343F
:1043F800234343601278032A02D00A78032A03D1A0
:10440800426880231A434260426803239B041A438C
:1044180042600B780122D2051B48002B03D11B4BAD
:104428001B78032B19D0C3689343C360164A184BF3
:104438004032D360FF2581351561164C5461164B07
:104448009361114B80335D609C60144CDC60144BAD
:1044580003600978002903D006E0C3681343E4E742
:1044680001680123194301600E4909780E4BC906FA
:10447800C90BC91881630D48D06130BD40F00040B8
:104488004C0AFF1F4B0AFF1F800003404A0AFF1F08
:10449800C00B00207A3E6A07000089040080890466
:1044A800CC240000480AFF1F250800002FFCA601A5
:1044B800F8B505004A484B4B4B4C4C4A4C4934D054
:1044C800022D32D086155710066286699E43B318AE
:1044D80083612078002833D00F6146480863464836
:1044E80000780122120380184861414E404C434B2A
:1044F800803E403C002D27D06521414AC9024148F1
:10450800012D2ED0022D31D0032D5AD0042D58D094
:104518003D49691831603D49A1602360E06002218E
:104528000846FDF703FC3A482BE0802606628669B8
:104538009E430123DB04F61886612078002801D009
:104548000A61CAE70B61C8E7324830600020A06002
:1045580023603148E06003210846FDF7E7FB2F4858
:104568000FE02F4B3360A2602160D7E72C4B5B1C18
:104578003360A2602160E06002210846FDF7D6FBA7
:1045880028482061F068FF210843F06026486061F0
:104598002648A0612648E0612648206226486062D5
:1045A8002648A0622648E0622648206326486063C1
:1045B800E020012D0DD02168022D0ED0814321600D
:1045C800F8BD224BEB183360214B73602160A26069
:1045D800A4E7216881432031F1E781434031EEE7C8
:1045E800C000034000001C004B0AFF1F000004002D
:1045F8008000034003000001440AFF1F00280B004D
:1046080055555537D6BE898E0080064255555500FA
:10461800805508220080067807EE753680660822E5
:104628000180063D80450822A49C5C544C444342CA
:1046380041524C46403A342E28007F554F49433D5D
:1046480037312B4C46403A342E28221C00800698DD
:10465800545A9850F0B5224B214D21498026204AC2
:104668000727BF04403BC03DE0248039022816627A
:10467800966914D0BE430127BF04F6199661194AFA
:104688001278002A1ED07A101A6101281ED0164A04
:1046980080182860154808610868A04314E00120C4
:1046A800BE43C004361896610E4A1278002A00D01C
:1046B800401018610E4828600E4808610868A04339
:1046C800403001E01F61E0E70860F0BD0848401E87
:1046D8002860094808610868A0432030F4E7000012
:1046E800C00003404B0AFF1F00800698805508222F
:1046F8000280063D804508228066082210B50A49D6
:1047080000200870094902200870FFF745FE084894
:10471800007800F011F8074C2078FFF7C9FE2078E0
:10472800FDF70AFB10BD00004B0AFF1F4C0AFF1FD4
:10473800480AFF1F490AFF1FF0B51A4A0323072535
:10474800D60019499B026024ED0157693F281AD009
:10475800B74305263604BE195661CA689A43CB1476
:10476800D218CA60CA69A2432032CA61CA69AA4378
:10477800CA610D4940398A6BC0061205120DC00B7B
:1047880002438A63F0BDB7430126B604BE195661D9
:10479800CA689A43CA60CA69A243CA61CA69AA4375
:1047A8008032E5E700F00040C0000340F8B53A4B1E
:1047B8005D6A9C6A00265E629E62384B58630E20D2
:1047C80018629E155E62402098625020D862FF20D1
:1047D8002B30586231484030012915D080210162C0
:1047E8002F49FF232D48A533403083602D4B43606C
:1047F8002A4B2D48403B18617D20C0000090471E81
:10480800009705D33846FAE7066225498331E8E779
:10481800264889050F18214840388763234B5B1CBD
:10482800C918816322480090224800780300FDF7E8
:1048380069F905040408060D08001F4800E01F4830
:1048480000901F4810601548403005E01D48F7E704
:10485800C16AC943890F14D000994B1E0093F7D23F
:104868000E4940398F630D4900228A62CA6282600C
:104878004E620A62FF2041304862074845628462FE
:10488800F8BDC16A104B1940116011680122090C6A
:10489800120489184160E3E70010034080000340D8
:1048A800CA0200002020000080560C206465210008
:1048B800102700004A0AFF1F204E00003075000034
:1048C80000002020409C0000FFFF3F3F00B5002172
:1048D800022000F021F80C49801C087000214220B9
:1048E80000F01AF80949801C08700121022000F024
:1048F80013F80749801C08700121422000F00CF8C9
:104908000449801C087000BD440AFF1F450AFF1FA8
:10491800460AFF1F470AFF1FF8B53B4C394A226079
:10492800394D394A07239B04803540320129A9694A
:104938000ED0994301239B04C918A9613349D1605A
:1049480033490B780121C905324E002B07D009E005
:1049580099430123DB04C918A9612F49EFE733788C
:10496800032B14D0D3688B43D36050630E2010629E
:1049780000275762FF201530506228480090307891
:104988000300FDF7BFF80507070D090B0D00D368F5
:104998000B43E9E7224802E0224800E02248009061
:1049A8000098431E0093FBD2686B57620002000E0A
:1049B80017621E4BD360FF23413353626523DB022A
:1049C80023601B4D2F78E023012F0AD02D78022D6C
:1049D80025680AD09D4325600D4B1B78002B07D016
:1049E80009E025689D432035F5E79D434035F2E70A
:1049F8003378032B03D0D3688B43D360F8BDD368D7
:104A08000B43FAE710000300400003407F407300A7
:104A18004B0AFF1F4A0AFF1F7F4053001027000060
:104A2800204E000030750000409C000040401000FF
:104A3800490AFF1FF8B5614C60688030806880F3D0
:104A48000888FDF77FF95E485E49006802258842BC
:104A580006D00020FDF7B6F868070169A94301618F
:104A680000F0D6F858480078FDF766F9574E002050
:104A7800F061F561564D75610120FDF77FF803205F
:104A8800F061FDF799F80746FCF7D6FF0646FDF7F3
:104A980093F850490860FFF731FE4F480068874295
:104AA80001D9381A01E0381A401E4C49884200D909
:104AB800084061688A8DD20709D0494A030C1268F8
:104AC80080B2534350431B02000A18180BE0C2017E
:104AD8008300D21A4300D21AC3001818921C8030DF
:104AE8009208400A1018E061FF313E4801314968D8
:104AF800006809183C480068081A41198B083B48A7
:104B08008A073B4903600D68920F52190A60042A0C
:104B180004D95B1C9207920F03600A60E169354F64
:104B2800C8183946FDF724F802463348334D036860
:104B3800D31803602A688A182A60BA4206D95B1C0F
:104B4800036039461046FDF713F82960FDF700F9B0
:104B58002B480078002810D0FCF76EFF294AE1693D
:104B6800801B12680B18934202D2511A091A01E0ED
:104B78007D21C9001548FDF7F1F8234D287A002852
:104B880011D0FCF759FF811BE3691048EA685C18EB
:104B98003C30A24202D9D21A511A00E01B49FDF753
:104BA800DDF800202872FDF7DFF80220FCF74AFF45
:104BB8000020FDF707F8FDF7DDF8F8BD0851FF1FE5
:104BC8000C0AFF1FB6412103490AFF1F00100040CD
:104BD800C4090000100AFF1F340AFF1FFFFF3F002F
:104BE800380AFF1F1C0AFF1F200AFF1F240AFF1F85
:104BF800280AFF1F710200006008FF1F2C0AFF1F10
:104C08001C09FF1FE408FF1F740BFF1FDC050000D1
:104C1800F8B5FEF723F8FDF7BBFD0120404E0090E4
:104C28003078404C022810D0FCF7C6FF05463220E9
:104C3800FCF7A4FFFDF752FE0F20FCF79FFF30782A
:104C4800012808D0FDF7F4FE1AE037484068006AEA
:104C5800FCF794FF24E033484038C06B4007400F0E
:104C6800012802D10020FDF78BF86068FF27013783
:104C7800B84360600220FCF781FF606838436060D9
:104C8800FCF79AFFA84201D3401B01E0401B401EDD
:104C980025491E2288615043244A49688018C86102
:104CA800244923480860234823498030C163FF21F1
:104CB800413141623078FDF763F820492048FDF71B
:104CC8004DF81F481F491430FDF748F80420FDF738
:104CD8000FFD1420FDF70CFD1520FDF709FD172029
:104CE800FDF706FDFF20FDF715F80120FDF74EF84A
:104CF800FF20F530FDF750F85820FCF7F1FE124878
:104D0800FDF750F80098FDF753F80720FDF756F81F
:104D1800E0690E490840FF300930E061F8BD000045
:104D28004A0AFF1F40F000400851FF1F72060000AA
:104D38000180063D000003403408000071020000B5
:104D480014100040FFFF3F003075000000FEFEFF1A
:104D580010B5072801D9062010BD04490870FDF7D1
:104D680033F804490248C861002010BDB04DFF1F48
:104D7800D11DFF1F4003FF1FB04DFF1F1C52FF1F17
:104D8800880100007A27FF1F1C52FF1FB04DFF1F2C
:104D98006C0400006419FF1F384FFF1F1C52FF1FCF
:104DA800942900008A27FF1F32FF32021488212825
:104DB80005145902E0013204123BA30108990B6261
:104DC800031A1802121D2B90014C2D107C02114958
:104DD8002DA47A0211105A16102D704EFF1F105A6A
:104DE80024104B24541069205A71205A2610CBF0F5
:104DF8004D205A72205A2C102AF82013020229C476
:104E0800011CA994DAB8945AD4541A2E10A9301A4D
:104E18001C1029DB1A8C20B2201A60182FD95E02C8
:104E2800112D5F300A1F1270DAD4705AEE701ACE44
:104E38001829104BE0581069705AF420E9305AD0FC
:104E480030DAE2301AFC20911911920763FFFF1A39
:104E58001802121D2A903DF1BF010203040506BA8B
:104E6800BA010FF9D93901B9E0CB4C7BE04BDD4FE2
:104E7800A01A3F182910DA54205ADE205A4120CBB4
:104E88002376F05ADF205A4320DA68405AE0205A45
:104E98004520DA59205AE1205A4720DA5E205AE2A2
:104EA800205A49201A6308EA12E799E0DA88404B49
:104EB800B450405A86404BE658101A1C2032031A48
:104EC800BC202C40787D1B0111A91512F712057220
:104ED8000BD2FF22B42A2802143075A049021112FD
:104EE800081508E001F09A10023A5002290A63D026
:104EF800071A0F6012051C307507141201CA815574
:104F08000111E91FA80D952D0211252E0211F93660
:104F180002111CBAFFB60112400DE1750211396980
:104F28000211556802112B747C0809143400000022
:040000051FFF18F9C8
:00000001FF
